:1000000000800020BD0100006139000019390000A6
:100010001939000019390000193900001939000098
:100020001939000019390000193900006139000040
:1000300061390000193900001D3000002131000035
:100040006139000061390000613900006139000048
:100050006139000061390000613900006139000038
:100060006139000061390000613900006139000028
:100070006139000061390000613900006139000018
:100080006139000061390000613900006139000008
:1000900061390000613900006139000061390000F8
:1000A00005190000111900006139000061390000D4
:1000B00061390000613900006139000061390000D8
:1000C00061390000613900006139000061390000C8
:1000D00061390000613900006139000061390000B8
:1000E00061390000613900006139000061390000A8
:1000F000613900008544000061390000CD4F0000E7
:1001000061390000094A00006139000061390000CE
:100110006139000061390000613900006139000077
:100120006139000061390000613900006139000067
:100130006139000061390000613900006139000057
:100140006139000061390000613900006139000047
:100150006139000061390000613900006139000037
:100160004D0C0000292100006139000061390000B8
:100170006139000061390000613900006139000017
:100180006139000061390000613900006139000007
:1001900061390000613900006139000061390000F7
:1001A00061390000613900006139000061390000E7
:1001B000613900006139000061390000564B4CF292
:1001C000205210B51A804DF628121A8000BF00BFC9
:1001D00003F0CAFB514B4FF010621A60504A9A600C
:1001E000504ADA60504A136813F4807304D14F49BF
:1001F0000B604FF4A85313604D4B1A78110703D5C9
:100200001A7842F008021A704A4B4B492A221A7097
:100210004A4A4B4B8B4204D252F8040F43F8040B6A
:10022000F8E7484B484900228B4202D243F8042B9E
:10023000FAE74649464A002352F8230041F82300D2
:1002400001336F2BF8D1434B434A802103F8011B44
:100250009342FBD1414B3D4A1A60414B8A221A70AE
:10026000A3F5805324225A70A0221A709A7992071B
:10027000FCD59A79D406FCD43A4A937903F00C035E
:10028000082B384BF9D103221A7140225A719A79FE
:100290009006FCD5334A9179324B4906FBD5324A58
:1002A000324911600221516020221A709A7902F0BD
:1002B0000C020C2AFAD12E4B2E4A1A602E4B2F4AD2
:1002C0001A6000225A60072243F8042C2C4AC3F813
:1002D0000C2D62B603F038FD144B1B68DA0705D508
:1002E000284803F0C5FC284B284A1A60284B1B7885
:1002F0005B0609D5244C254B22689A4204D121483B
:1003000003F0B6FC0023236005F090FB03F032FB02
:1003100003F060FAFEE700BF0E2005403080044085
:10032000823F04000100002B10D0034014D0034092
:1003300002D0074000E00740E0A4FF1FC8A500006E
:10034000308EFF1FE0A4FF1F5C0300200084FF1F0E
:100350000000000000E400E05FE400E008ED00E0E1
:100360000050064000400640448004400000030165
:1003700004800440C010050014E000E0FF76010096
:1003800000002020B9E276611CE00340A5C3945A26
:1003900000F00740FFFFFFFFFFFFFFFFFFFFFFFF32
:1003A000FFFFFFFFFFFFFFFFFFFFFFFFFFFFFFFF5D
:1003B000FFFFFFFFFFFFFFFFFFFFFFFFFFFFFFFF4D
:1003C000FFFFFFFFFFFFFFFFFFFFFFFFFFFFFFFF3D
:1003D000FFFFFFFFFFFFFFFFFFFFFFFFFFFFFFFF2D
:1003E000FFFFFFFFFFFFFFFFFFFFFFFFFFFFFFFF1D
:1003F000FFFFFFFFFFFFFFFFFFFFFFFFFFFFFFFF0D
:10040000FFFFFFFFFFFFFFFFFFFFFFFFDEF9FFFF23
:1004100010B5054C237833B9044B13B10448AFF33E
:1004200000800123237010BDE0A4FF1F0000000026
:10043000C4A50000084B10B51BB108490848AFF32C
:1004400000800848036803B910BD074B002BFBD0A0
:10045000BDE81040184700BF00000000E4A4FF1FE3
:10046000C4A50000E0A4FF1F0000000042F2212309
:10047000984200D1704702460149024802F016BF77
:10048000449D0000208FFF1F38B50121092003F093
:1004900007FC0121092003F0FDFB5149514B524A51
:1004A000524C09685248216000251D70158002F0E9
:1004B00097FC40F2836003F009FD2946C022201D0D
:1004C00005F01EFE00F0CCFD102003F06FF828466A
:1004D00003F046F84FF48064102003F09BF8013CD1
:1004E0000544F9D12A1EB8BF02F2FF3292124149E7
:1004F0004148424D02F0DAFE4FF48071012000F0D5
:10050000A7FA642003F0D2FB112003F083F86424DF
:10051000112003F07FF82B68384A1844013C28600A
:10052000F6D1374B374C83FB0013C017C0EB631376
:100530001020136003F06EF804F54255204604F5D0
:10054000C27401F08BFCA542F8D14BF6803000F06C
:10055000EBFC00F0FFFA102000F066FB00F07EFBE1
:1005600000F03AFC41F2883004F064F8092003F00E
:1005700017F9254C254D20600A2003F011F9244B72
:100580002860014640F2DC5201201A6000F060FA57
:100590002A68204940F6B83303FB02F3002BB8BFAA
:1005A000FF331B12072000F0BFFB22681A4940F6F8
:1005B000B83303FB02F3002BB8BFFF3307201B1235
:1005C00000F0B2FB206828B94FF48071BDE83840D4
:1005D00000F03EBA0146BDE83840002000F038BACD
:1005E000108FFF1F24D8FF1F10DAFF1F0082FF1F8C
:1005F000F099FF1F589D0000208FFF1F1C8FFF1FC9
:100600001F85EB5100A5FF1F20D8FF1F148FFF1F70
:10061000188FFF1F6C9D0000809D00002DE9F043A6
:10062000274D284E2C783368C4F340049C4283B095
:1006300005D022462449254802F038FE3460244E75
:100640002C78336804F001049C420AD022462149E8
:100650001E4802F02BFE84F00101092003F01AFB72
:10066000346004F0D5FA002823DD1B4D1B4E2B68A7
:1006700001935028A8BF5020DDF80480184F814610
:10068000002407E02B680093009BBA68C8EB0303C3
:10069000934211D2C4EB0901301904F0C7FA0444A3
:1006A000A1450F49EED8002C03DD21460B4804F08C
:1006B00009F903B0BDE8F08301230B73F3E700BF32
:1006C00074020020B0D9FF1F949D0000208FFF1FEF
:1006D0000CD8FF1FA09D000050010020BCD9FF1FB7
:1006E000249BFF1F70B5154D04F020F92B68834241
:1006F000044601DB3CB970BD02202C6003F0D6FA41
:10070000312CF7DC70BD0E4E4FF480723046002164
:1007100005F0F6FC3F2C224606F10101A8BF3F225E
:10072000084802F0F1FD03463046194600F8013B47
:1007300000232B60BDE8704004F0E4BAB4D9FF1F79
:100740000CD7FF1F289AFF1F08B5FFF767FFFFF7B9
:10075000C9FFBDE8084001F077B900BF0FB4F0B59C
:10076000C3B048AB02AC53F8046B019332464FF46C
:100770008071204607F076FB204605F041FF0E4AC7
:10078000019B118897782152251832464FF48071C9
:100790002046AF7007F066FB204605F031FF0146AA
:1007A000204603F06BFD054802F068FD43B0BDE84C
:1007B000F04004B0704700BFAC9D0000208FFF1FC9
:1007C000704700BF00B583B002F0A2FF044A054B9A
:1007D00012680192019A1A6003B05DF804FB00BF31
:1007E00050010020ACD9FF1F002070470368C9B238
:1007F0001B6818470368C9B21B6818470368C9B269
:100800001B6818470368C9B21B681847F0B40F4C3F
:100810000F4823680F49104A104F114E114D367979
:1008200001332360036803F59663036082B00B68AD
:100830000193019B10681B1A3B600B680093009B9F
:1008400013602E7002B0F0BC704700BFE8ECFF1FD1
:10085000ACFFFF1F5001002010D8FF1F08D7FF1F5B
:1008600018DAFF1F1F80004008B5084603F0FCFCA3
:10087000012008BD08B5084603F0F6FC012008BDBC
:1008800038B508460D4605F0BBFE0446014628462D
:1008900003F0F4FC204638BD10B508461446114656
:1008A00003F0ECFC204610BD03F0C6BD08B50846B9
:1008B00003F0B2FC003018BF012008BD08B508469F
:1008C00003F088FC003018BF012008BD084611461F
:1008D00003F01CBC084603F053BC00BF084603F0FD
:1008E000F9BB00BF03F094BB4B0803F1376000F580
:1008F000D830B0FBF1F003F0E9BA00BF10B54B08F7
:1009000003F13760144600F5D830B0FBF1F003F086
:10091000DDFA2046BDE8104003F04EBB03F074BD85
:1009200003F03EBD03F02CBD03F00CBD03F016BD7B
:1009300010B5044602F0F6FA204610BD704700BF1D
:10094000034B82B01B680193019802B0704700BF4F
:100950005001002070B5334CE37A0546EBB172B616
:10096000E37AD9071A4606D52F49E268086802409B
:10097000A2610A601A469B0706D52C4923690868BC
:10098000E27A0340E3610B60560705D5284A6369A4
:1009900011680B402362136062B62368254AD96848
:1009A000914206D0244E254825491E60DA60186120
:1009B000196000210A202D0103F06CF945F00C05A7
:1009C0002368EDB24FF00042DA625D63DA6A002A12
:1009D000FCDA4FF0004100229D6BD9625A63DA6A5B
:1009E000002AFCDA01210A209E6B03F053F9E37A16
:1009F0000C49F6B21A4683B1D80703D5114A896962
:100A000011601A46990703D50F4BE169E27A196024
:100A1000530702D50D4B226A1A60280200F47F406A
:100A2000304370BDF099FF1F80E100E084E100E0F9
:100A300088E100E00110013801403F000110017819
:100A400000003F8000E100E004E100E008E100E098
:100A5000F8B50C460501FFF77DFFA04259D0E0052F
:100A60002F48C37A48BF45F00105EBB172B6C37A8F
:100A7000D9071A4606D52B49C2680E6832408261F2
:100A80000A601A469F0706D5274903690E68C27A8D
:100A90003340C3610B60560705D5244A436911688A
:100AA0000B400362136062B60368214AD968914221
:100AB00006D0204F204E21491F60DA601E61196068
:100AC0001F49EDB210264FF000420E60DA625D63FE
:100AD000DA6A002AFCDAE4B24FF00042996BDA627B
:100AE0005C63DA6A002AFCDAC27A16499B6B0C4C0A
:100AF00010230B60134662B1D10703D5124BA169D5
:100B000019601346920705D45B0702D50F4B026AA2
:100B10001A60F8BD0E4AC169C37A1160F4E700BFDC
:100B2000F099FF1F80E100E084E100E088E100E04F
:100B30000110013801403F000110017800003F80A2
:100B400088F00F4084F00F4000E100E008E100E091
:100B500004E100E0094A0A4913680A48F0B443F482
:100B60008053094E094D0A4C1360C0270022082308
:100B700037702A702370F0BC086070472C800440E6
:100B8000348FFF1F28DAFF1F21C00C4000C00C402B
:100B900001C00C40F0B41C491C4B0A791A700B6858
:100BA0001B4A1A6002259D800A791A48186102F1D1
:100BB000804202F50432184EDE6040F20110D88007
:100BC0004FF4166400200627B026DC829D60DC838B
:100BD00098829F839861107016700A790F4B1048A5
:100BE0001A7053119B0003F1604302F1100403F5E6
:100BF000614302F01F0201210A4D40F8245001FA1E
:100C000002F21A60F0BC704718DAFF1F1A80004029
:100C100028DAFF1F00C00C4040EDFFFF1B800040A2
:100C20000084FF1F0D080000172808B503DDA0F1A0
:100C30002203032B07D8C0B202F0ECFC024A13686F
:100C400043F04403136008BD20B00340024A136818
:100C500023F040031360704700600340F0B4144871
:100C6000144B02791A700368134A1A6000219980A4
:100C70000279124C1C6102F1804202F5043240F20A
:100C80000116DE804FF4166502240D4FDD82A82682
:100C9000DD839C609F619C829983D960094C1170AF
:100CA000094B1670027921601A70F0BC704700BFC2
:100CB00020DAFF1F1A80004010B00340ECECFF1F49
:100CC00040EDFFFF14DAFF1F1B80004008B5064A05
:100CD000064B12791A70FFF7C1FF0549054B00203A
:100CE000082208701A7008BD18DAFF1F1A80004029
:100CF00000C00C4001C00C40024B1B68D88A80B277
:100D0000704700BF20DAFF1FC0B2054B012253F825
:100D1000303011B183F80021704783F8802070478C
:100D2000DCA10000704700BF0EB400B5C2B043ABF9
:100D30004FF4807153F8042B019302A807F092F846
:100D400002A805F05DFC014602A803F097FA0448EA
:100D500002F094FA42B05DF804EB03B0704700BFB4
:100D6000208FFF1F38B50E4C0E49020284FB02345F
:100D7000D217C2EBA4140546024623460620FFF70D
:100D8000D3FF002D0BDDB4F5807F21464FF000002E
:100D9000A8BF4FF48071BDE83840FFF759BE38BD99
:100DA000F1197605309E000010B5094C094903027F
:100DB000024684FB0304DB17C3EBA414234606207E
:100DC000FFF7B2FF21460120BDE81040FFF740BE0B
:100DD000F1197605509E0000F8B540F2836003F0EB
:100DE00075F841F2883003F025FC404B4049414AF8
:100DF0004148424D4CF220544DF628171C8042F2D7
:100E000010761F800024D1232E8004800B80148054
:100E100003F0A4FA3A4902463A4802F047FA04F0CD
:100E200001F8394902462046FFF77EFF374B1B7811
:100E30009B0656D40121062002F032FF0121022038
:100E400002F02EFF0121032002F02AFF01210420DD
:100E500002F026FF0121052002F022FF01210220DD
:100E6000FFF752FF01210320FFF74EFF012104206D
:100E7000FFF74AFF01210520FFF746FFC82002F0D7
:100E800015FF00210220FFF73FFFC82002F00EFFF0
:100E900000210320FFF738FFC82002F007FF0021E0
:100EA0000420FFF731FFC82002F000FF00210520D9
:100EB000FFF72AFF01210A2002F0F2FE144B154829
:100EC00010221A6001F08CFF134B186808B9134BFD
:100ED0001868FFF747FF124B1868BDE8F840FFF7A6
:100EE00063BF10490220FFF71FFFA3E70E20054054
:100EF000002005401620054004200540062005403E
:100F0000709E0000208FFF1F8C9E000000F00740A5
:100F100084F00F40F099FF1F20D8FF1F188FFF1F8C
:100F2000148FFF1FA49E0000F8B5104D104F2C68C1
:100F3000104E114B93FBF0F344F480042C600246F6
:100F40005C1E012038600D4934600620FFF7ECFE7E
:100F50000B4B0C4A0C48002548F6A37440F20111D3
:100F60001D601C6018601160F8BD00BF3C8004402B
:100F70000C60034004600340006CDC02C49E00006F
:100F80000060034010600340A28F01002E4B1B68DD
:100F900013BB70B582B016460D46044600F0C2FF82
:100FA000B0B1621B40F6E44303FB02F3002BBCBF6D
:100FB00003F57F43FF331B14B3F5486F2CDC272B5D
:100FC00034DDA3F5C862B2F5487F0AD802B070BD1F
:100FD000002EE6D102B070BD1A461C490720FFF76B
:100FE000A3BE1B4D1B4A2C681B4904FB03F382FB69
:100FF0000324DB17C3EBA414224604EB44040720AC
:1010000004EBD474FFF790FE601040F6B8339842BA
:1010100014DD2B60184604E00D4A40F6B83318463C
:10102000136002B0BDE87040FFF79CBE00932246FB
:101030002B460A490720FFF777FEC7E76328D8BF8A
:1010400064202860EDE700BF20D8FF1FE49E000069
:10105000188FFF1FF1197605309F0000FC9E0000DD
:10106000704700BF10F0FF0F14BF034B034B10225B
:101070001A600120704700BFC4F00F40C8F00F4055
:10108000F8B50D4F0D4E0E4D0E4C02F041FB38469B
:10109000002101F0E3FE32462946384604F084FC84
:1010A0002046002101F0DAFE324629462046BDE8FE
:1010B000F84004F079BC00BF18DAFF1F0C8FFF1F47
:1010C0003109000020DAFF1F2DE9F04F93B0FFF740
:1010D00013FE504B1B68002B60D14F4D2B68002B2B
:1010E0005FD1B0F5966F59DC4C4A4D49DFF8548119
:1010F0004C4F4D4ED1F80090D7F800E0D8F80010D2
:1011000034684FF4166000FB03204FF0000A00F52E
:10111000166C0246D3461388C9EB0303734522F8C5
:10112000023BC4BF9E464FF0010BA342BCBF1C460E
:101130004FF0010A94451944EDD1BBF1000F65D180
:10114000BAF1000F60D1394C394A23681268C8F8E7
:10115000001003F5966323604FF496613ABBFFF7E6
:101160002FFB344B34483A683168DFF8DCB01A6042
:101170000160FFF7E5FBDBF80030DFF8ACA0DFF83B
:10118000A490C01A42F20F72904213DC2B68B3FA9B
:1011900083F300225B092B603A60326013B0BDE834
:1011A000F08FB0F5966F9FDA13B0BDE8F08F00F0C6
:1011B00067FED6E7FFF7C4FBDAF80030D9F8002065
:1011C000CBF80000D8F80010206891FBF0F1072060
:1011D00000911A49FFF7A8FDD9F80030DAF800208D
:1011E000174902A805F0E0F9D9F80000FFF79AFDC9
:1011F0000023DAF80010D9F80000C8F800301A46C9
:101200002360FFF7C3FEC1E734609CE7C7F800E046
:1012100096E700BFF8FFFF1F14DAFF1FECECFF1F7B
:101220001C8FFF1F28030020300300202C03002008
:10123000308FFF1FBCFFFF1FB8FFFF1F4C9F000038
:101240006C9F000034030020B0FFFF1F0369D3F838
:101250003402D3F83032C01A704700BF0369D3F8A4
:101260003012D3F83422914208D2D3F83022511CE4
:101270001A44C3F8301292F8300070474FF0FF3034
:10128000704700BF0369D3F83012D3F8342291427B
:101290003DBFD3F830229B1893F830004FF0FF3059
:1012A000704700BF704700BF0369D3F83C24B2F514
:1012B000007F03D30123037100207047D3F83C243F
:1012C00010B49C180132C3F83C2484F83812012071
:1012D00010BC7047F0B40569D5F83C34B3F5007F15
:1012E0001FD2D5F83C64D5F83C44C6F5007696424A
:1012F00005F50E7302D20127324607714AB1013C4F
:1013000023448D1811F8014B03F8014FA942F9D17C
:101310000569D5F83C341344C5F83C341046F0BC9C
:10132000704701230371F0BC0020704738B5036992
:101330000A4A026093F84024022A044601D020465B
:1013400038BDD3F85C54002DF9D0284601F0EAFDF1
:101350002846082102F044FB204638BD989F000033
:10136000F8B5C16887680D783B78DBB203F02002DE
:10137000EDB212B313F0100F90F8523477D0022B65
:1013800000F0D28090F85234032B00F0CD8090F81A
:101390004934012B00F0D18190F84934DBB2022BA3
:1013A00000F0028290F84934042B00F087818023FA
:1013B0003B70C36802221A70F8BD02F0FF06EA060D
:1013C000044623D405F0400202F0FF0012BB03F0F4
:1013D000100303F0FF06002B7CD015F0010540F050
:1013E0006281D4F83824D4F83C349A4207D2D4F835
:1013F00038345A1C2344C4F8382493F838522369EB
:101400001D70A368D0221A70E16868E010236F068F
:101410000B7028D594F849340A2B00F0DA8005F0D7
:10142000040505F0FF03002D5CD0A3680021D02245
:10143000092084F84904C4F83C141A702269D4F8CD
:10144000581413785B0884F84A3409B18847226934
:10145000D4F83C34002B00F02E8194F838621670DA
:101460000123C4F83834E36802221A70F8BD022B55
:1014700000F0888090F85234032B00F08380D0F87D
:101480003432D0F84C240233934200F0078190F8B4
:101490004934042B00F0FD80D0F8343201339342FC
:1014A00080F0D58090F84934042B00F0CB80D0F840
:1014B00034320269591CC0F834120344127883F89C
:1014C000302090F84934042B00F02E81C3680222AA
:1014D0001A70F8BD94F849340A2B00F044810223B5
:1014E0000B70F8BD94F8422484F85034012A00F0BF
:1014F0006B81002A00F06281022A00F09381032AA6
:1015000000F00D81A368C0220A20002184F849045C
:10151000C4F834121A7023691B785B0884F84A34C3
:10152000E36802221A70F8BDD0F85C2413689B8B24
:101530001C0603D590F85234022B78D090F8523420
:10154000032B52D0BA4B12791C68012393402342DB
:10155000C5D0B84BB8491A70D0F85C2412790A701B
:101560000023E90680F8523440F1D780C268122186
:10157000072480F849441170826880211170C0F8F6
:101580003834F8BDD0F85C341A68928B120603D553
:1015900090F85224022A3FD090F85224032A00F0F7
:1015A0009480A34C1A79246801239340234296D057
:1015B000A149A04B0A70D0F85C2412791A70826895
:1015C0000023802180F8523480F849341170C168BA
:1015D00085E7D4F85434002B3FF421AF0022C4F83F
:1015E0003022D4F83402984719E70B781D06FCD551
:1015F000924B12791A70002380F85234D0F83C34A0
:101600000269013BC0F83834D0F83834034493F809
:1016100038321370C16862E7864A1B791370836899
:10162000E8221A700323C16880F8523457E7814BCF
:1016300012791A708368F0221A700323C16880F847
:1016400052344CE790F85134002B3FF430AF90F80F
:1016500049240023042A80F8513401D080F8493409
:101660008368B0221A70D0F834320269591CC0F86D
:1016700034120344127883F8302090F84834012B58
:101680007FF41FAF2023013BFDD1836880221A70B5
:1016900017E790F85134002B7FF4FEAEE8233B703F
:1016A000D0F84C24F8E6C0233B702369E1681B782E
:1016B00084F8490413E784F83832D0E690F84834C7
:1016C000012B4DD0B0233B7000E75C4A1B791370AF
:1016D000002380F8523490F84924042A18BF80F877
:1016E00049348368B0221A70D0F84C340269013B47
:1016F000C0F83432D0F83432591CC0F834120344E4
:10170000127883F8302090F84834012B05D120233B
:10171000013BFDD1836880221A70C168DFE6484929
:101720001F2002F0E5F9EDE690F85134002B7FF42C
:10173000CDAE012380F85134C8E605F0100303F064
:10174000FF02002B46D115F0010551D080F852243C
:10175000D0F83834002B40F08F80052380F84934CE
:1017600080233B70B2E694F8422484F85064012A46
:1017700000F09280002A78D0022A00F09480032A98
:1017800000F0A48023691B78D4F83422B2F5007FDE
:10179000DBB2BFF4A4AED4F83422A0180132C4F8EE
:1017A000342280F830309AE6EC0632D4E9074BD583
:1017B0000522802380F849243B7087E603222149D3
:1017C000112002F095F99DE603221E49122002F035
:1017D0008FF997E600231222072480F8523480F80C
:1017E00049440A70826880211170C0F83834F8BD0D
:1017F000D0F838340133C0F83834D0F83C24934260
:101800003ED390F8483480F84954012B7FF45AAF06
:10181000A6E70722122380F849240B7083688022F0
:101820001A70F8BD032206491E2002F061F969E62C
:101830002C8000401F8000401E8000401C80004023
:10184000D1190000C519000090F85224012A31D0A6
:10185000D0F84C34012B0CBFE823E023032280F89E
:1018600049243B7003691B7830E623490322112089
:1018700002F03EF9E16885E7062380F849346FE716
:1018800090F85234012B27D0D0F838340269034441
:1018900093F83832137019E617490322122002F028
:1018A00027F9E1686EE7154903221E2002F020F9AE
:1018B000E16867E7E12280F852343A70D0F85C249E
:1018C0000F4B12791A7003691B78FFE50B491F2033
:1018D00002F00EF9E16855E70222F12380F8522464
:1018E0003B70D0F85C24064B12791A70036990F8AB
:1018F00039221A70EAE500BFC5190000D1190000AD
:101900001B80004000210148FFF72ABD388FFF1FD0
:1019100001210148FFF724BD9C93FF1FC3681B787A
:1019200003F02003CBB903F0FF0290F84234012BFF
:1019300010B5044680F8492427D053B3022B32D087
:10194000032B37D0D4F85434CBB10022C4F8302262
:10195000D4F83402BDE81040184790F850340133F1
:10196000DBB2012B80F850340AD990F84234012BB5
:1019700024D093B1022B13D0032B18D0704710BD85
:1019800090F84134012BF0D1F8E7122002F02CF945
:10199000D8E7112002F028F9D4E7112002F024B989
:1019A0001E2002F021B91E2002F01EF9CAE71F20F6
:1019B00002F01AB91F2002F017F9C3E7122002F053
:1019C00013B900BF00210148FFF7A8BF388FFF1FE0
:1019D00001210148FFF7A2BF9C93FF1F2DE9F843A7
:1019E000134BDFF85C90DFF85C80124E124D1E60E6
:1019F00000244FF47A774A4641461C711C739F605D
:101A000018465C731D6103F0CFFF0C4B4FF0010EC5
:101A100005F264451C711C7383F80DE04A4641468B
:101A200018461D619F601E60BDE8F84303F0BCBF0F
:101A3000D4FFFF1F989F0000388FFF1FC0FFFF1FBC
:101A40000C8FFF1F2D1300002DE9F0473F4C84B091
:101A5000FEF776FF236842F20F72C31A934221DC2D
:101A60003B4CFFF731FB206801285BD0E368384A24
:101A7000012B60D0374C23682BB1374A374B1268A3
:101A80001B689A4202DA04B0BDE8F0870020FFF735
:101A9000E9FA334A00232360136004B0BDE8F0473D
:101AA000FFF714B92F4E304FDFF8D080DFF8D09019
:101AB0002E4B3168DFF8A4C03A68DFF89CA01B68A1
:101AC000D8F80050D9F800E0DCF800C0DAF800A03F
:101AD0002060BEF1000FB8BF0EF1030E002DCAEB5F
:101AE0000C00B8BF03350290AD104FEAAE00019074
:101AF00000951F48FEF732FE0023C9F80030C8F8F1
:101B000000303B60336072B61A4B4AF202614BF20E
:101B1000804219801A8062B60D4CFFF7D5FA206812
:101B20000128A3D10023A1682360FEF791FFE36899
:101B3000074A012B9ED154690F4D002321461846B8
:101B40002C60D360FEF784FF94E700BFECFFFF1F1B
:101B50000098FF1FF0FFFF1FACFFFF1FB4FFFF1F28
:101B6000F4FFFF1F1CD8FF1FFCA4FF1F14D8FF1F8A
:101B7000B49F00000C20054020D8FF1F80D5FF1F18
:101B80000CDAFF1F2DE9F8435FEA90082B4D4BD08C
:101B9000DFF8C890DFF8C8C0012600224FF6F97EB2
:101BA00039F822302C6803F500410132043BC1F3BF
:101BB0000F11671C734598BF002690452F602CF8C5
:101BC0001410EDD1002E2FD11D4E33680446FBB109
:101BD0001C4A1D481D490368184E013303600868FC
:101BE0002044086013681A4C434413602B68B3F513
:101BF000166F04BF0023336023683BB92B68B3F52D
:101C0000707F03DDFEF7C6FF01232360BDE8F88384
:101C1000104B5B6873B110490A4A00230120306001
:101C20000B6013602B60D4E72B68C8EB03032B60B9
:101C3000BDE8F8830120FFF715FAECE7E8FFFF1F86
:101C4000F4FFFF1FB4FFFF1F1CD8FF1F80D5FF1F2D
:101C5000F0FFFF1F0098FF1FACFFFF1FC482FF1F94
:101C600028DAFF1F38B51649164B0A681B68164C50
:101C7000013284FB0304DB170A60C3EB241472B641
:101C8000124B1D68C5B1294651F8042B1A6062B683
:101C90000F48224601F0A6FD72B60E4A0E4913689F
:101CA0000868286001330D60136062B60B4A136840
:101CB00023441360204638BD62B6C02038BD00BF43
:101CC000FCA4FF1F1898FF1FD34D621084D5FF1F7F
:101CD0000482FF1F14D8FF1F28D8FF1F0CDAFF1F34
:101CE0002DE9F0418CB006784578837890F8038030
:101CF0004779007991F803E0CDF800800C4602970F
:101D00000190A078CDF818E094F801E005902078D3
:101D10000390CDF810E0E07994F806E00A9060793D
:101D2000CDF824E094F804E0089031462A46204893
:101D3000CDF81CE0FEF712FD212E03D000200CB0E0
:101D4000BDE8F081312F12D0322FF7D1B8F1010F59
:101D500026D0B8F1020FF1D1012DEFD161782378AF
:101D6000144A03EB0123936015602846E7E7B8F1B6
:101D7000010F0DD0B8F1020FE0D1012DDED1617855
:101D800023780C4A03EB01235361D5602846D6E73C
:101D9000012DD3D1074B22781A61DD602846CEE7AA
:101DA000012DCBD1034B22785A601D602846C6E72F
:101DB000F09F00000098FF1F2DE9F043047846785B
:101DC0008378C5784779007985B088460190009579
:101DD00091462146324602971E48FEF7BFFCA12CD1
:101DE00003D0002005B0BDE8F083012D14D0022DF2
:101DF000F7D1812E1FD0822E25D0832E14D0842E91
:101E0000EFD10122002388F8002088F80130022356
:101E1000C9F800300120E5E70F4B5B6888F8003017
:101E20002846C9F80050DDE7FF22002388F800208B
:101E300088F80130EBE7084A0023926888F8002010
:101E400088F80130E3E7002388F8003088F8013093
:101E5000DDE700BF28A000000098FF1F10B472B695
:101E6000054A064913680C68046001330860136072
:101E700062B610BC704700BF14D8FF1F28D8FF1FE0
:101E80002DE9F047244D2B68182B33DDDFF890E067
:101E9000224EF046B146841E00F65E174FF0000C4D
:101EA00072B6DEF8000038B32A680368C8F800305C
:101EB000531E2B6062B600F1080300F1C80A2246E7
:101EC00032F9021F23F8041CB2F9001023F8021C97
:101ED00004335345F4D1C0F800C072B632680AB971
:101EE00013E01A461368002BFBD1106062B6603411
:101EF000BC42D5D1BDE8F08762B672B6306840B159
:101F00000368C9F8003062B6D5E7C9F8000062B6C8
:101F1000EDE762B6BDE8F08714D8FF1F84D5FF1F38
:101F200028D8FF1F0120704770B584B072B6194BD6
:101F3000194D1A48702241260F2480211A702E70E4
:101F40001A460470197013781B06FCD5144B1868D8
:101F500062B6144B144C984298BF00EB800001A964
:101F600098BF40000A2201F03DFD01A92046002350
:101F700011F8012B01333AB10A2B20F8022FF7D1C7
:101F80001623237004B070BD5B00DBB2237004B075
:101F900070BD00BF00000240070002400600024082
:101FA000080002407F969800D899FF1F431E072B18
:101FB00014D872B60A4951F8230068B170B4094CBC
:101FC000058834F81320466841F82360521B24F832
:101FD000132062B670BC704762B67047002070472D
:101FE000640000203C030020013807280BD872B69B
:101FF000074B53F8203043B100205B680130002BC1
:10200000FBD162B67047002070471846F9E700BF61
:10201000C8000020F0B5864672B6022201231C4992
:102020001C4F02E0294601330132072B01F1010563
:10203000F9D0097817489C00090744F0010605D536
:1020400057F8341069B157F83610C1B1092AE9D1EF
:1020500062B6114B00221A707046BDE8F04002F0E3
:1020600075BD0D490D4D0A7840F8345000EB43130F
:102070000EF10800013A58600A7062B6F0BD0649D8
:10208000074B40F836300A7800EBC603F0E700BF94
:1020900048A000000080FF1F1101002088004000C0
:1020A000C8004000431E072B1DD81B4A400140F0CA
:1020B000100030B4104472B6184CE25C032A1BD8EE
:1020C000DFE802F00212151703220D88E25410F027
:1020D000080F14BFC823882343EA0543083103606F
:1020E000416062B630BC704708300222EDE705223D
:1020F000EBE708300422E8E7094A52F8230038B138
:10210000084A52F82300416042F8231062B6E9E71A
:1021100042F82310034AF7E70080FF1F2001002048
:10212000C8000020E80000202DE9F04FDFF850A3A0
:10213000DFF850B389B049E0DFF810834FEA930924
:1021400008EBC905013C6A68E4B2052CA2F108005D
:1021500000F02581062C00F04181072C00F056810B
:102160001F0700F13D8158F839301B0C99B222F855
:10217000081C002B00F02981AC4E56F82470002377
:1021800022F8063C42F8043C002F00F01F82A84FC2
:1021900057F824305860A74E47F8240036F814301A
:1021A000194426F8141002F0B1FC002800F0078250
:1021B000A14AA24B15F0080F00F1080018BF134602
:1021C000686048F8393008238AF800309AF80040EF
:1021D000E4B262071AD59A4B1B78A3B199490A78E1
:1021E00002F0FF0322B1013BDBB20B7003B900BE6A
:1021F00095490A7802F0FF032AB1013BDBB20B706C
:10220000002B00F0B28104238AF8003004F00803A8
:1022100003F0FF02002B00F046819BF80030DBB298
:102220001C0989D19E08894C54F8363004EBC6024B
:10223000C3F38303013B51680C2B00F28480DFE879
:1022400003F086868282828282824E8282820700A8
:102250007F4A0B680092784A4968DFF8089244F890
:10226000362000277A4A7B4D276198B20126A76164
:10227000C9F80030C9F80410176007972E70FEF7F0
:10228000F5F8B9F80030B3F5086F00F0318340F28B
:102290002B8142F22132934200F0828200F21D82B1
:1022A00040F60132934200F0EA8200F23682B3F542
:1022B000106F00F03E8340F68122934240F003828B
:1022C000B9F804300796042B00F05184052B40F038
:1022D000FA81614A614B12781A70012262E25C4B0A
:1022E00000931B684BB3DFF8A0E15A4D5C48BEF881
:1022F000002029780678402A174646F0020C28BFAD
:102300004027002981F001012970A2EB07020CBFD0
:102310008821C82104EBCC0592B286F0010641EA7F
:1023200007416B60AEF8002044F83C103B44067057
:10233000002A00F00D81009A13604A4B1A88B2F50A
:10234000A06F00F00981484A012313703BE7454B19
:102350001A8842F221039A4200F04C814148FFF76B
:10236000BFFCA8B13E483B4D03782A7883F00101B9
:10237000002A43F0020301700CBF8821C82144F8F1
:10238000331004EBC30382F0010200212A7059606C
:10239000294B354A44F836300123137013E71907E7
:1023A0007FF5E1AEFFF75EFC00283FF40CAF85F04F
:1023B000080500042D4B2E4A6B6040F08000286019
:1023C000537983F001035371FDE61B4A1B4B15F053
:1023D000080F18BF134648F83930F4E61B0778D5C4
:1023E00002F0B4FB234A224E52F82430002B00F0B6
:1023F000F1805968305D42F8241003F108026A60E8
:10240000032845D8DFE800F0A1429E9B1E077FF518
:10241000AAAE85F00805184A6A60184B144A2B606A
:10242000D37983F00103D371CDE600BF64000020AF
:10243000000000203C030020C8004000880040004D
:102440001C01002085000020650200200080FF1F85
:10245000FCFFFF1F84000020B8D9FF1F14010020DB
:102460001001002008010020942007400482FF1F73
:1024700020010020C80000200082FF1F8000030010
:102480008020074090200740200000200222325583
:102490001A8815F0080F0CBF8823C82343EA0243AB
:1024A00048F839308FE6E00762D4210600F1CD808C
:1024B000A20706D5A24AA34913780220DBB2137003
:1024C0000870E30602D59F4B10221A7009B0BDE8D0
:1024D000F08F58F83900000CFFF754FB9A4A9B4BD9
:1024E0006A6048F839306EE640F20232934200F0FA
:1024F000D58100F2B480B3F5817F00F0E48100F271
:10250000DA80802B00F00F82822B40F0DC80B9F85B
:10251000043003F07F03082B00F2D5808C4A8D49EC
:102520009B001A440F704F701378980748BF01231F
:102530004FF0020248BF0B700792864B32E1042233
:102540003255A5E705223255A2E7032232559FE70F
:10255000402F18BF0023EEE600219A7859707E4B79
:102560001A707E4A012313702DE602F0ABFC4AE696
:102570007B4B7A487B491A614FF0020E80F800E0ED
:10258000734F0A707849196099606D4E6D4D724CA9
:102590009A610D213970FF213170DFF800E2297056
:1025A0002270724D724A8EF800109F27012406F89F
:1025B000047C5D600470DA6009B0BDE8F08F6D4A9C
:1025C00048F83900137801331370FCE546F824000D
:1025D000694FE0E5335D032B00F24A8101A252F816
:1025E00023F000BFC7210000C7210000A92600007A
:1025F000A3260000614B08784A7818705A708878D2
:10260000CA789870DA7008791A6818714879587120
:10261000862A8879987101F1070148D05148584DB0
:1026200003782A7883F00107002A43F00203077039
:102630000CBF8820C82044F8330004EBC30382F0A9
:10264000010200202A70586088E641493D4B8022F3
:102650000D2008701A70A2077FF533AF2AE7B3F593
:10266000A06F00F09D8040F23D82A3F5D063012B66
:1026700029D8444A536833B3B9F80200B9F8046062
:1026800002E00C325368F3B111888142F9D15188CC
:10269000B142F6D1000A03280CBF1A7812890792BA
:1026A00080E0012333558EE5002333558BE5364B0F
:1026B0000F221A70B2E740F22112934206D040F284
:1026C0002122934202D0224A0F231370234A01236E
:1026D0001370224A0123137075E548F2A122934238
:1026E00000F0168100F20B8148F2A112934200F033
:1026F0000F8148F2A2129342E5D1B9F80630022BBD
:10270000E1D92248FEF72AF8124B8022BB211A7029
:1027100003229F705970079244E042F221029342D3
:10272000D4D042F221229342CDD11949194A1A4BF1
:102730000968116099F802201A70079A3B4631E047
:102740008820074080200740C482FF1F8000C0000F
:10275000C020074014010020982007409420074023
:102760000080FF1F1001002088004000240000208E
:102770008800002011010020000000204C030020F0
:102780008400002050A0000085000020BCA00000B4
:102790005001002054030020740200208C200740C8
:1027A000079A0023B9F80610B64895F800E00778B4
:1027B000DFF8D48291423CBF0A460791402A114675
:1027C00028BF4021BEF1000F47F002090CBF882648
:1027D000C82604EBC90C46EA014644F83960521A8F
:1027E00087F001068EF00109CCF8043006700B4426
:1027F00085F8009019D140297FF468AF46F00206B1
:1028000004EBC604A04963601404B9F1000F24D19D
:1028100044F0880441F8364085F800E0077013441E
:10282000402A7FF453AF002212E0402AE6D946F056
:10283000020608EBC6014B60B9F1000F16D09349B0
:10284000934C48F8361084F800E0403A0770403363
:10285000904900980A80036038E744F0C80485F87E
:1028600000E00770134441F83640D9E78A49E7E7AA
:1028700015F0080F0CBF022303233355A3E4B9F866
:102880000430042B00F04C81052B7FF41CAF834BEC
:10289000B9F802201A70079A3B4683E7B9F804108A
:1028A00001F07F0108293FF60EAFB9F80230002B86
:1028B0007FF409AF7A48079A89000844017841F00B
:1028C000020101706EE7B9F8041001F07F010829D8
:1028D0003FF6F9AEB9F80230002B7FF4F4AE704841
:1028E000079A89000844017821F00201017059E734
:1028F0006C4A6D4B117807963246197052E748F2D0
:10290000A132934204D048F2A14293427FF4DBAE5D
:1029100007AA65496548FFF74FFA00283FF4D3AE90
:10292000079A614B3EE7604B02221F705F7007926F
:1029300038E7554E5B4A99F80230137006F58077F8
:1029400002E00836B74207D0336A1B06F9D5706A31
:10295000083802F0FBF8F4E7554901915549564A09
:1029600002915649564F574E0595002303978846C6
:102970001D4617460496386828B1466802F0E6F806
:102980003046002EF9D1019B186800233B60039B61
:102990001A46002342F8253028B1466802F0D6F8DE
:1029A0003046002EF9D1019A98F8003011460022E5
:1029B0000A60029A1146002241F8042F049A0291FB
:1029C000023B4FF0000122F81510032B07D8DFE877
:1029D00003F0810281024FF0010388F80030019B6F
:1029E00001350433082D07F10407019308F10108AC
:1029F000C1D1354B3548059D029519460023344A0F
:102A000003704FF0020801270D4613E0BE0046F0A8
:102A1000020E46F003060023082F44F83E301A4801
:102A200044F8363000F0A980B8F1090F57D00137CB
:102A300008F1010815F8013B02F8043B072F00F0EC
:102A4000A6801E07E2D5019202F060F8019A0028E4
:102A50005DD004EB4713BE00083058600E4B44F8BD
:102A60003630019202F052F8019A002845D046F023
:102A7000010304EBC30E0830044944F83310CEF8C8
:102A80000400C4E7100100200080FF1FC8004000C0
:102A9000840000202000002088004000B8D9FF1FDB
:102AA000C02007401C010020140100200801002064
:102AB000C8000020E4000020640000202001002065
:102AC000000000203C03002048A00000110100206D
:102AD000C42007404FF0000388F800307FE7029DD4
:102AE000079A5FE640F2213293423FF4EFAD40F2A5
:102AF000214293423FF4EAADE5E52D4B2C491B788A
:102B000046F0010E013344F83E000B707FE7284B7E
:102B100027491B78BE00013344F836000B70A0E74C
:102B200099F80230234A1370002B3FF439AE224E3D
:102B3000224B96F80580A3F10807B8F1000F18BFE3
:102B40001F463B6813F080037FF42AAEB02219467B
:102B50001B48019388F0010803F0D2FA194A184B78
:102B60007B603A6086F80580019B079A1AE6114A55
:102B7000154B12781A70324614E600EBCE06134A53
:102B8000134F40F83E20029D7760079A0AE6114BEA
:102B90001148C4F8E430C4F8EC300023C4F8E00075
:102BA000C4F8E800C4F8F030C4F8F8303FE700BFDC
:102BB0001101002018D8FF1F20010020D880FF1F1E
:102BC0000482FF1F8000B000140100208000030079
:102BD0000082FF1FC482FF1F8000C0002DE9F84360
:102BE000204CFFF7A1F9002204F5847023461A60F7
:102BF0005A60083383424FF00001F8D11A4A1B4F44
:102C000013681B4D1B481C4EDFF87880DFF878C036
:102C1000DFF87890DFF878E043F480231360C4F3A2
:102C200007233B70C4F307432B70240EFF2302F5E8
:102C300028320470114D88F8003011488CF80030AB
:102C4000D4323370012389F8003070268EF80010DA
:102C50004FF40074102107F8183C2E7004601170B6
:102C6000BDE8F8830080FF1F348004409C200740AB
:102C7000B0200740B42007401020074049E400E09E
:102C800008E100E0802007408820074094200740AA
:102C90000021074010B4047F4160022CC26002D0C2
:102CA00010BC00F059B9836810BC1847F0B4464B0B
:102CB000464A186BDC6A01791170454922790A701D
:102CC0009A6A00790870002A46D05968C9688A4211
:102CD0003ED82168CC8B240402F1FF3065D4C0F3C8
:102CE0000E00C883C88B80B2C882196B0968C88B74
:102CF000000452D4C2F30E00C883C88B002480B2F3
:102D000012F1FF32C88218BF01229C62D96A2E4894
:102D100009680D6800F12404A54236D00068C46833
:102D200014F0804F0C680D6815BF24882478023594
:102D3000013544F000440D604463196B254B09795B
:102D40001970214912B1CA6A12791A70F0BC704721
:102D5000521A9A620122D9E7586B196805681E4C0D
:102D60000A63CC62CC682D681C4E24F08044032793
:102D7000B542CC6083F825701FD1037F4260022BDF
:102D8000C2601ED0F0BC00F0E7B8016890F82400E3
:102D9000CC6840F000404863CFE7CC8BC2F308001A
:102DA00004F47E442043C883A7E7CC8BC0F308001B
:102DB00004F47E442043C88394E72B461146F0BCBC
:102DC00018478368F0BC1847F099FF1F1F80004028
:102DD0001C8000401B80004000000FFF952C00006D
:102DE00090E80C00F0B41C6859682568164F174E1F
:102DF00029432160164D17491760D660156111608F
:102E0000417A154A5C180A3194F8244053F821504D
:102E100002EBC40149680D60017A5C1803EB810183
:102E2000247ECD6902EBC40149680D60817A58188F
:102E300003EB810390F83000596B02EBC002F0BC49
:102E400053681960704700BF01401F00011000382F
:102E50000110007800001F80DCA10000F0B572B600
:102E600099B902688AB103790F2B0ED8274C2188B3
:102E700041FA03F5ED070AD503F1007303F59063FA
:102E8000B2EB431F03D162B6F0BD204C2188002372
:102E900041FA03F212F0010207D00133102BF7D1EF
:102EA00062B6002203710260F0BD01259D402943F6
:102EB000218062B6164E174D174FDFF864E0D9B285
:102EC0000171346844F0020434602C6844F0020458
:102ED0002C60A6F580268224A5F5802503F10073D9
:102EE0003C6003F59063223E243D0C4C8EF80010AC
:102EF0005B0131702970217003601A605A609A601A
:102F0000DA601A615A619A61DA61F0BD2801002025
:102F1000408004403C800440008000401F8000400E
:102F20001A80004003790F2B11D8094A10B413708E
:102F300072B6084904790A880123A34022EA0303F0
:102F40000B8062B61022002310BC02710360704730
:102F50001A8000402801002010B4EFF3108272B6EE
:102F6000437F33B9017F012907D003290FD0012303
:102F7000437702B962B610BC7047124C2168A1B108
:102F8000114943610B68836108605861EFE70F4C9A
:102F9000216881B10E4943610B6883610860586103
:102FA0000C4B4FF080511960E1E7074B41618161A3
:102FB00020601860DBE7064B41618161206018608A
:102FC000EEE700BF3C010020380100202C0100206A
:102FD0003001002004ED00E070B5EFF3108272B60E
:102FE0000C4C206880B10C4E00254369236073B1FE
:102FF0009D6102B962B6457783689847EFF3108206
:1030000072B620680028F0D102B962B670BD336094
:10301000EFE700BF2C01002030010020FFF7DCBFEC
:10302000184A30B41468002C27D0036821688B42FA
:103030000ED2CB1A00218460C1602360E060106072
:103040000223037530BC704711688B42144608D3C5
:10305000A2685B1A0360002AF6D18260C460A06097
:10306000EEE7D268C2608460E060C568CB1A0222D5
:10307000A8602360027530BC70478460C460106033
:10308000DEE700BF34010020F8B5224E34682CB3CF
:103090002368002B3AD1204F1D4604E03468ECB180
:1030A0002368002B32D1A36803B1DD60206933604F
:1030B000036825751B68BB4221D1037F4560022B45
:1030C000C46020D0FFF748FF6368002BE6D0236080
:1030D0002046FFF7A5FF3468002CE1D1EFF3108301
:1030E00072B60E4A00211068116003B962B628B1A9
:1030F0008468FFF795FF20460028F9D1F8BD2246E5
:1031000000219847E0E783689847DDE7013B2360AB
:10311000E4E700BF34010020952C000044010020AA
:10312000024A136801331360FFF7AEBF500100205D
:1031300008B5084601F0BCFB012008BD08B50846EB
:1031400001F0B6FB012008BD38B508460D4603F076
:1031500057FA04460146284601F0B4FB204638BD24
:1031600010B508461446114601F0ACFB204610BDD0
:1031700001F038BC08B5084601F07AFB003018BFF2
:10318000012008BD08B5084601F050FB003018BF0B
:10319000012008BD0846114601F01EBB084601F09B
:1031A00043BB00BF084601F0FBBA00BF01F0BEBA46
:1031B0004B0803F1B76000F55840B0FBF1F001F0A7
:1031C00039BA00BF10B54B0803F1B760144600F5DB
:1031D0005840B0FBF1F001F02DFA2046BDE8104058
:1031E00001F078BA01F0E6BB01F0B0BB01F09EBB84
:1031F00001F07EBB01F088BB0368064A1B6893425E
:1032000005D110B5C8B201F053FB012010BDC9B201
:10321000184700BF3D3100000368064A1B6893420F
:1032200005D110B5C8B201F043FB012010BDC9B2F1
:10323000184700BF3D3100000368064A1B689342EF
:1032400005D110B5C8B201F033FB012010BDC9B2E1
:10325000184700BF3D3100000368064A1B689342CF
:1032600005D110B5C8B201F023FB012010BDC9B2D1
:10327000184700BF3D310000704700BF00B5064A47
:10328000036812885B6883B001A9ADF804200222AC
:10329000984703B05DF804FB9CA1000010B50368DB
:1032A00014465B689847204610BD00BF0EB400B5B9
:1032B00082B003AA52F8041B019204F08DFD02B003
:1032C0005DF804EB03B0704770B50E4D82B02B680B
:1032D0000093009E044608E001F018FE2B6801935D
:1032E000019BA2689B1B934207D2236820465B691F
:1032F00098470028F0DB02B070BD4FF0FF3002B0FD
:1033000070BD00BF50010020F8B50D46A1B11646B2
:1033100082B10746002404E00134A64205F8010BFF
:1033200008D03846FFF7D0FF0028F5DA01233B73B9
:103330002046F8BD3046F8BD0846F8BD374A384942
:1033400013681B06FCD40B6813F08003F8D172B627
:1033500034490A78002A5FD0334A3448F0B4344CF8
:10336000176806682568D4680C303E44143200683B
:103370001268304F35442C4420440244C2F34E02BC
:103380002D4E2E482E4D2F4C42F400423A603768A5
:1033900006682D682C4A24680C303E440068126888
:1033A0002A4F35442C4420440244C2F34E02284E96
:1033B0002848294D294C42F400423A603768066893
:1033C0002D68274A24680C303E4400681268254F57
:1033D00035442C4420440244C2F34E02224E23487A
:1033E000234D244C42F400423A60376806682D6849
:1033F000214A24680C303E440068126835442C444D
:1034000020440244C2F34E021C4842F400420260CF
:103410000B7062B6F0BC704762B6704724B00340D0
:1034200024B00B404901002038B003403CB00340B9
:1034300040B003402CB0034058B003405CB00340A0
:1034400060B0034064B003406CB0034030B0034050
:1034500038B00B403CB00B4040B00B4044B00B4088
:103460004CB00B402CB00B4058B00B405CB00B4044
:1034700060B00B4064B00B406CB00B4030B00B4000
:1034800030B42948294A2A4B2A4D6024E12104708E
:1034900011701B78284C082B30D00A2B274828495C
:1034A00037D00C2B0CBF35223D2212232A6023601B
:1034B00002600B60234B24491B78244ABBB10123D3
:1034C0000B601360224B23491B78234A012B26D91A
:1034D000042B0FD9082B1ED9102B94BF86238723CA
:1034E0000B6013601D4B01221A7030BC70470B60DB
:1034F0001360E7E784230B601360F3E700F58E2089
:103500000F490830012213232A60236002600B60F8
:10351000D0E73922F7E785230B601360E2E78023C9
:103520000B601360DEE700BF00400740014007402A
:10353000389AFF1F08B003400CB0034008B00B409E
:103540000CB00B404C01002020B0034020B00B40D9
:10355000399AFF1F24B0034024B00B4049010020DA
:1035600068B10E4A1378C3B90D490978012010706B
:1035700019B10C490C4A0B601360FFF781BF074B70
:103580001A7852B1064A18701378002BF5D0054A04
:10359000054B10601860FFF773BF70474C010020A7
:1035A0004901002024B0034024B00B400C2830B463
:1035B00017D91023984228BF18461C46104A114DAF
:1035C0001178181A8C42287018D00F4913700B7894
:1035D00023B10E490E4A00230B60136030BCFFF785
:1035E0004FBF0A2802D90C231C46E7E7082802D956
:1035F0000A231C46E2E708231C46DFE730BC70477D
:10360000389AFF1F480100204901002024B00340E0
:1036100024B00B4028282FD8334B2DE9F0411E5CF5
:10362000FF2E2BD0314B1B78002B2AD132062CD405
:1036300072B62F4D2F4C2F46012326602B7062B699
:1036400072B623681B060CD43B781BB9F4E72B78C1
:10365000002BF1D062B601F059FC72B6236818064F
:10366000F5D5254B1B6800222A7062B6234A1078D4
:1036700043FA00F0BDE8F081002070470020BDE86B
:10368000F081FFF75BFE3206D2D572B61C4DDFF833
:103690007C801C4C06F04007FFB206F03F06D8F8CD
:1036A0000030DFB123F01003C8F80030012326609A
:1036B000134A2B7062B672B6236819060CD41378BD
:1036C0001BB9ECE72B78002BE9D062B601F01EFCA9
:1036D00072B623681B06F5D50B4BC3E743F0100306
:1036E000C8F80030E2E700BFA0A1000049010020B7
:1036F0004B01002000B0034010B0034048010020FF
:103700004A01002000B00B4010B00B400CB00B4041
:10371000F0B51B4B1B4E596818689A68DB6885B07A
:103720006C460FC4337899071DD5174A174C137888
:10373000174913F0700318BF1370164A164B8027F1
:10374000177000263320032226706D4608701A7009
:1037500072B6043C45F001052046A84762B62378BE
:1037600013F0700309D10D4B064901E0013B02D073
:103770000A78D207FAD505B0F0BD237005B0F0BDC8
:10378000CCA1000001000240000002400400024001
:103790000B000240070002400A000240410D0300F6
:1037A000B0F5006F0AD210B5094B1B78DB07044651
:1037B00006D504F1A0500078C0B210BD00207047BB
:1037C000FFF7A6FF04F1A0500078C0B210BD00BF03
:1037D0000100024008B5FCF757FEFCF7B5FF01F009
:1037E00095FBFAE7844641EA000313F003036DD129
:1037F000403A41D351F8043B40F8043B51F8043BB4
:1038000040F8043B51F8043B40F8043B51F8043BBA
:1038100040F8043B51F8043B40F8043B51F8043BAA
:1038200040F8043B51F8043B40F8043B51F8043B9A
:1038300040F8043B51F8043B40F8043B51F8043B8A
:1038400040F8043B51F8043B40F8043B51F8043B7A
:1038500040F8043B51F8043B40F8043B51F8043B6A
:1038600040F8043B51F8043B40F8043B51F8043B5A
:1038700040F8043B403ABDD2303211D351F8043BFA
:1038800040F8043B51F8043B40F8043B51F8043B3A
:1038900040F8043B51F8043B40F8043B103AEDD2A9
:1038A0000C3205D351F8043B40F8043B043AF9D2FA
:1038B000043208D0D2071CBF11F8013B00F8013BCD
:1038C00001D30B8803806046704700BF082A13D3DA
:1038D0008B078DD010F003038AD0C3F10403D21AF2
:1038E000DB071CBF11F8013B00F8013B80D331F826
:1038F000023B20F8023B7BE7043AD9D3013A11F8A6
:10390000013B00F8013BF9D20B7803704B78437010
:103910008B7883706046704708B5104C08E02368C8
:1039200059050DD423681A050FD42368DB0411D47C
:1039300023685803F3D5FEF7F7FB23685905F1D543
:1039400000F0A0FD23681A05EFD501F03FFB2368C6
:10395000DB04EDD501F058F8EAE700BF34800440FD
:1039600008B5FFF7D9FF00BF014B10221A8070473E
:1039700000200540704700BF094908B50B6830B109
:103980006A461844A2F58052904202D20860184656
:1039900008BD02F045F80C2303604FF0FF3008BD6E
:1039A0003C9AFF1FEFF3138070B9EFF310836BB9EC
:1039B000EFF305825AB94FF48070EFF311832BB106
:1039C000984228BF184670474FF0FF3070470F2AC3
:1039D00001D81846F1E7014BD05CEEE7F0E300E0D8
:1039E00002F054B8F0B44D1E2E46002400E001341D
:1039F000B0FBF2F302FB1300092800F130078ABF85
:103A00003730F8B2C0B206F8010F1846002BEED1DD
:103A10000A1953704CB1107815F8016F28700133F2
:103A2000E01A834202F80169F5DB0846F0BC7047F2
:103A3000704700BF10B40F4B53F8302092F880420B
:103A40002CB1012369B182F8803010BC704703EBC0
:103A5000C0035B681A6841B922F002021A6010BC08
:103A6000704782F8003110BC704742F003021A60C0
:103A700010BC7047DCA100001C4A02EBC003012906
:103A80005B6811D004291BD052F83000002280F866
:103A9000802229B1022920D0032922D01A60704740
:103AA0004FF480721A60704752F830004FF4A272DF
:103AB00080F880121A601A6822F020021A6070479B
:103AC00052F830104FF4A272012081F880021A607F
:103AD0001A6842F020021A60704740F203121A601E
:103AE00070474FF481721A60704700BFDCA100007C
:103AF000212848D8F8B5042A44D8DFE802F0484B1A
:103B00004E0345004FF410262B4B03EBC0030D462C
:103B10005C68216811F4E06148D0284B284A2949A3
:103B2000C3F89C2104F140422748C3F8A411A2F530
:103B30009221264FC3F8A0017C292548C3F8A8711B
:103B4000C3F8AC012CD9A2F594237C2B2AD9A2F579
:103B500096237C2B28D9A2F598237C2B29D9A2F572
:103B60009A227C2A27D81B4872B6236823F4702334
:103B700043F08072C4F384011643236040F821505F
:103B8000266062B6F8BD70474FF43026BCE74FF4AC
:103B90000026B9E74FF44026B6E74FF42026B3E7F6
:103BA0000D48E1E70D48DFE70D48DDE7FFF764FF6B
:103BB000B3E70C48D8E7F8BDDCA100000084FF1F84
:103BC000E18EFF1F898EFF1FB58EFF1F5D8EFF1FC9
:103BD000318EFF1F189BFF1F409AFF1F789AFF1F0F
:103BE000C89AFF1FF89AFF1F1A4B03EBC00010B4CE
:103BF000426802F14043A3F592217C2923D9A3F521
:103C000094217C290DD9A3F596217C291FD9A3F5F0
:103C100098217C2919D9A3F59A237C2B11D80E4C15
:103C200000E00E4C72B613680D4823F08773C2F3A0
:103C3000840123F4803343F08073136044F821003F
:103C400062B610BC7047074CECE7074CEAE7074C3C
:103C5000E8E700BFDCA10000189BFF1F789AFF1F58
:103C6000313A0000409AFF1FF89AFF1FC89AFF1FC1
:103C700030B4054B054D064C002210211A602A6015
:103C80002060196030BC704714D0034004D003405A
:103C900000D00340212801D8FFF7CCBE704700BFF9
:103CA000212801D8FFF7E8BE704700BF2DE9F8438F
:103CB000054672B6204F214B214A1B683C681268AA
:103CC00062B6520102D5322B88BF013495B3C3F5D9
:103CD000BB331C4EDFF86490DFF86480FF334FF491
:103CE0007A72A6FB031302FB04F404EB931472B67E
:103CF000D9F800103A68D8F800E062B6C1F5BB33D5
:103D0000FF33A6FB03031EF0806FC4EB93134FF445
:103D10007A7002D0322988BF013200FB0233B3F53A
:103D20007A7F04D3013D05D004F57A74DFE701F012
:103D3000EDF8DCE7BDE8F8835001002018E000E072
:103D400004ED00E0ABAAAAAAF8B52D4B2D49DFF887
:103D5000D0E0DFF8D0C02C4E2C4D2D4C2D4A2E4FEC
:103D60004FF4000018604FF0807018604FF0007042
:103D700018604FF0806018604FF0006018600020FD
:103D8000086028234BF6FF71CCF80010CEF8003005
:103D9000336013602B6023603B60B362936209223F
:103DA00045F8242CC4F8D80F05F57F65C7F8D41F53
:103DB00007F5FF2707F5FA67C6F8F83F2B6006F509
:103DC000FF26C4F8D42F05F5FD2504F5FF2438603F
:103DD00006F2F4761148316005F5FF6504F5FD64DF
:103DE0002B6023600260FFF74BFB1920FFF75EFF9B
:103DF000FEF7F4FE40F21310BDE8F840FFF756BF9F
:103E000008E100E004800340148003402480034064
:103E10002C8003401C8003403480034000800B4012
:103E20000C800340088003402DE9F84F214B1B68AC
:103E300007460BB101221A70DFF888901E4D99F8E1
:103E40000040DFF884801D4E01343F2C8ABF4FF0C4
:103E5000000A5FFA84FA5446AB462B78A34216D187
:103E6000FFF7A0FD40281FDC33791B06F5D59BF832
:103E7000003001333F2B86BF00221346DAB218F818
:103E80000330DBB2F3712A702B78A342E8D00C49DF
:103E90000A4BFFB208F804700120BC22087089F8B0
:103EA00000A0DA70BDE8F88FFF28D6DD01F02EF80B
:103EB000D3E700BFE4010020E101002000A006409C
:103EC000E0010020E80100205C0100202B4A2C4981
:103ED0001368F0B543F4806313600A78294F2A4EC3
:103EE0002A4D2B4C2B4900233B7033702B702370D1
:103EF0000B70002A3DD0152A21D0274B1B78012BAF
:103F000025D0052B30D01F2827D8002002460125B8
:103F1000224B234C1A7023495D7004224FF0020E8D
:103F200088273C26402598729A704FF4005083F8F9
:103F300013E05A751F74DE7025700860F0BD1A4BCF
:103F400040F213321A60144B1B78012BD9D1174B56
:103F50004FF451721F281A60D7D9C0F34432C0F30E
:103F6000471500F01F00D3E7114B4FF451721A6050
:103F7000C9E7104B40F213321A60BEE734800440A8
:103F80009C0100205801002059010020E801002078
:103F9000E1010020E0010020209BFF1F00A006405F
:103FA0002DE400E004E100E018C0044044A0044017
:103FB0001CC0044040A00440144B14499B7803F0FB
:103FC000EC0200F003031343420700F00F0248BF66
:103FD00043F01003042A8B7013D00C4B0B4A5B790F
:103FE000C10603F0EF0348BF43F010035371937908
:103FF000820603F0EF03054A48BF43F010039371B4
:1040000070478B7943F040038B71E6E700A00640D0
:10401000234B1B685B0541D510B5224C237823B197
:1040200000F074FF2378002BFAD11F481F4A204B61
:104030004FF4005400210460D1701B78FBB1152BA4
:1040400003D11C4B40F203121A601B4B1B7803F088
:104050007F03012B1DD0052B03D1184B40F2031217
:104060001A60174A114B1748174912681C79DB79F7
:10407000002303700B700AB10123137010BD134BA2
:1040800040F203121A600C4B1B7803F07F03012BE4
:10409000E1D10F4B40F203121A60E2E7704700BF14
:1040A00034800440E001002084E100E000A00640EC
:1040B0009C01002018C00440209BFF1F1CC004402E
:1040C00054010020580100205901002040A0044064
:1040D00044A004400A4A38B50546137803F0FF04AB
:1040E000002BFAD101212846FFF7DAFD21462846A8
:1040F000FFF7D0FD034A044B52F835201A6038BD53
:10410000E0010020DCA10000E401002009B140F042
:104110008000174A1378984216D010B4154C2468C2
:1041200064050FD503F07F03012B1CD0052B11D0A4
:10413000002900F07F0114BF6023442301290DD022
:10414000052902D0107010BC70470B4943F440732E
:104150000B60F7E7084B00241C60E9E7074943F4CC
:1041600040730B60EEE7054B00241C60E0E700BFE6
:10417000209BFF1F348004401CC0044044A0044026
:10418000104B1A7882420AD00F490968490505D5B3
:10419000AAB1152A09D068B1152801D01870704746
:1041A0000A4A40F213311160F8E7084A0021116011
:1041B0000028F1D1064A40F213311160EEE70449BC
:1041C0000A60E8E79C0100203480044018C00440E5
:1041D00040A004400D4B1B6813F4806305D02128D8
:1041E00005D90B4B00201860704718467047094BE3
:1041F00010B5074C53F8303023600121FFF750FD14
:10420000236800221A70012010BD00BF34800440D2
:1042100054010020DCA100000F4B1B6813F48063E5
:1042200008D0122808D0142811D00C4A537B03F070
:10423000FE03537300207047094B40F202321A60AC
:10424000064A537B43F00103537301207047054B2B
:1042500040F202321A60F3E73480044000A00640C6
:104260000CA0044014C00440034B1B685B0501D53F
:10427000FFF7DABD704700BF348004402DE9F84FE6
:10428000294B1B685A0548D5284B1B6805460BB1BE
:1042900001221A7005EB010A554540D2DFF89C80D7
:1042A000234CDFF89C90234F0AE015F8012B09F806
:1042B0000B20214A0123AA45137088F800602ED0F4
:1042C00098F80030227803F1010BBBF13F0F86BF55
:1042D0000026B3465FFA8BF69345E6D1BC22FA700E
:1042E00005E03A7913060BD422789345DDD1FFF728
:1042F00059FB4028F5DDFF28F6DD00F007FEF3E767
:10430000227801323F2A86BF00210A46D1B219F82D
:104310000220D2B2FA712170E6E7BDE8F88F054BB2
:10432000BC22DA70BDE8F88F34800440E40100203C
:10433000E101002000A00640E0010020E80100208B
:104340005C01002010B5044C237823B100F0DEFDA1
:104350002378002BFAD110BDE0010020064A074B5C
:104360001B781078DBB2C0B283422CBF3F3000F123
:10437000FF30C01A704700BFE1010020E8010020B3
:10438000054A064B10781B78C0B2DBB2984238BFA2
:104390004030C01A704700BF58010020590100206A
:1043A00030B4154B154C1A782378D2B2DBB29A424E
:1043B0001ED001333F2B0ED91149124B08781968D2
:1043C0000023C0B2237021B1D31A1A2B01DC0023C1
:1043D0000B7030BC70470A480A49C05C0968DDB2FE
:1043E000C0B225700029F4D09A4238BF4032EBE7C2
:1043F0004FF0FF30EDE700BF5801002059010020C9
:10440000A001002054010020084A094B12781B78B3
:10441000DBB29A4207D00133402B28BF0023054A64
:10442000D05CC0B270474FF0FF3070475801002099
:1044300059010020A00100200D4B1B685B0516D51B
:1044400030B40C4B0C4CDA780C480D4902F0CB021E
:104450004025DA705D74DA7842F03402DA7023783D
:104460000268DBB20B700AB10023137030BC7047D6
:104470003480044000A0064059010020540100206F
:1044800058010020F0B4384B1A7912F0300F2CD0BC
:1044900072B6997D01F0FF0200293DD062B6334F1C
:1044A000334938780D78334E1C46C0B2EDB2431C08
:1044B000402BE17928BF0023AB4202F1FF32C9B2A1
:1044C0001CBFF154184612F0FF02F0D12A4B1B68B2
:1044D000C2B23A704BB1A84236BFC5F14005401B8D
:1044E00040192728C4BF01221A701F49CA78D2B2C6
:1044F000150616D452060DD51B4B1B795B0609D544
:104500001E4B1F491B6800220A7003B11A70164B1C
:104510003C22DA70F0BC70474022D9795A7462B6F6
:10452000E3E70B791C06E5D5164B174E1C7833785C
:10453000E4B2DBB29C420ED0144D01E0A3420AD09B
:104540000133402B28BF00230879E85CC0B2C87152
:10455000087D0728F2D9DBB2034933700B791806BE
:1045600044BF7C23CB70C5E700A006405801002063
:1045700059010020A001002054010020E401002086
:10458000E0010020E8010020E10100205C010020A2
:104590002DE9F84F214B1B6807460BB101221A7019
:1045A000DFF888901E4D99F80040DFF884801D4E9A
:1045B0000134272C8ABF4FF0000A5FFA84FA544670
:1045C000AB462B78A34216D1FFF7ECF940281FDC4D
:1045D00033791B06F5D59BF800300133272B86BFB6
:1045E00000221346DAB218F80330DBB2F3712A70F6
:1045F0002B78A342E8D00C490A4BFFB208F80470AC
:104600000120AC22087089F800A0DA70BDE8F88FAC
:10461000FF28D6DD00F07AFCD3E700BF600200205F
:104620005D02002000C006405C0200206402002001
:10463000F40100201C4BDFF894C01A681B49F0B548
:1046400042F480521A4D1A60DFF884E0194F1A4E76
:104650001A4C00238CF800304FF451722B701F2835
:1046600040F213358EF800303B70337025600A60DD
:1046700012D819460124124A124D11701248547072
:1046800000212C27402693724FF40034917011744E
:10469000D7702E700460F0BDC0F34431C0F34714EE
:1046A00000F01F03E7E700BF348004400CC0044063
:1046B000F10100205D0200205C02002008C00440DF
:1046C00000C0064031E400E004E100E0F001002019
:1046D00064020020144B14499B7803F0EC0200F0B4
:1046E00003031343420700F00F0248BF43F01003D7
:1046F000042A8B7013D00C4B0B4A5B79C10603F074
:10470000EF0348BF43F0100353719379820603F01F
:10471000EF03054A48BF43F01003937170478B794C
:1047200043F040038B71E6E700C00640F8B5134B39
:104730001B68DB041FD5124C237823B100F0E6FB85
:104740002378002BFAD10F4B0F4A104D104F114E0A
:10475000114C12484FF4003119600023D37040F21D
:1047600003113960316029681579D279237003709B
:1047700011B101230B70F8BDF8BD00BF34800440B7
:104780005C02002084E100E000C00640EC01002053
:1047900008C004400CC00440F0010020F1010020DA
:1047A0000A4A38B50546137803F0FF04002BFAD106
:1047B00001212846FFF774FA21462846FFF76AFAD6
:1047C000034A044B52F835201A6038BD5C020020C1
:1047D000DCA100006002002009B140F080000F4A17
:1047E0001378984219D010B40D4C2468E40412D503
:1047F00003F07F03082B02D10A4B00241C60002920
:1048000000F07F0314BF60214421082B03D1054B26
:1048100041F440711960107010BC7047219BFF1F5C
:10482000348004400CC00440704700BF0D4B1B682F
:1048300013F4805305D0212805D90B4B00201860B4
:10484000704718467047094B10B5074C53F8303085
:1048500023600121FFF724FA236800221A70012047
:1048600010BD00BF34800440EC010020DCA100003A
:104870000C4B1B6813F4805306D00E2806D00A4A4E
:10488000537B03F0FE03537300207047074B064A27
:1048900040F202311960537B43F00103537301204E
:1048A000704700BF3480044000C0064004C004408C
:1048B000034B1B68DB0401D5FFF76ABE704700BFDE
:1048C0003480044070B5094E04464518AC4204F1EA
:1048D00001040AD03368DB04F8D514F8010CFFF7A3
:1048E00057FEAC4204F10104F4D170BD34800440A1
:1048F00010B5044C237823B100F008FB2378002B7B
:10490000FAD110BD5C020020064A074B1B781078D4
:10491000DBB2C0B283422CBF273000F1FF30C01A97
:10492000704700BF5D02002064020020054A064B6C
:1049300010781B78C0B2DBB2984238BF4030C01A42
:10494000704700BFF0010020F101002030B4154B8A
:10495000154C1A782378D2B2DBB29A421ED00133BA
:104960003F2B0ED91149124B087819680023C0B2A9
:10497000237021B1D31A1A2B01DC00230B7030BC39
:1049800070470A480A49C05C0968DDB2C0B22570A8
:104990000029F4D09A4238BF4032EBE74FF0FF30A5
:1049A000EDE700BFF0010020F10100201C02002013
:1049B000EC010020084A094B12781B78DBB29A42BE
:1049C00007D00133402B28BF0023054AD05CC0B27A
:1049D00070474FF0FF307047F0010020F1010020D8
:1049E0001C020020054B064A1B7806491268DBB200
:1049F0000B700AB100231370704700BFF101002053
:104A0000EC010020F001002030B42B4B1A79940601
:104A10001FD52A48DA790378294901333F2B0978D1
:104A2000C8BF00238B42D2B203D0264CD9B2E25485
:104A30000170254A116861B1244A1278D2B29342BA
:104A400036BFC2F140029B1A9B18272BC4BF01231B
:104A50000B70194AD378DBB2180611D45A060DD55B
:104A6000154B1B795B0609D5194B1A491B680022A7
:104A70000A7003B11A70104B2C22DA7030BC7047E8
:104A800011790906EAD5144910480C780178C9B2A1
:104A90008C420DD04A1C272A84BF00210A460F4DA4
:104AA000054C98BFD1B2AA5CD2B2E2710170D5E7D1
:104AB0006C21D170D2E700BF00C00640F001002099
:104AC000F10100201C020020EC0100205D0200200A
:104AD000600200205C02002064020020F40100203B
:104AE00000F0F4B800F07CB800F056B800F090B8D0
:104AF00000F0BCB900F096B90846114600F002B9C2
:104B0000084600F083B900BF704700BF72B60D4879
:104B10000268B2FA82F31D2B10DC4FF00041D9403D
:104B200022EA0102026062B6074803EBC303DB001E
:104B3000C2180021C15010465160704762B6002073
:104B4000704700BF349BFF1FBC85FF1F0D4B0E4AF3
:104B5000C31AA2FB03231B091D2B0CD80B4A127886
:104B600052B972B60A484FF00041026821FA03F3C5
:104B70001A43026062B67047064A1278002AF0D0E3
:104B8000FDF748BABC85FF1F398EE33811010020BC
:104B9000349BFF1F1C01002038B50F4D286878B1E9
:104BA00043880288C118013393420C7A02D24380B1
:104BB000204638BDFFF7CAFF002320462B6038BDD2
:104BC000064B1B782BB10220FDF7F0F92860002876
:104BD000E6D14FF0FF3038BD700200201C010020EC
:104BE00010B5094C206818B143881844007A10BDEC
:104BF000064B1B782BB10220FDF7D8F92060002866
:104C0000F2D14FF0FF3010BD700200201C010020D7
:104C1000044B054A1B6850881BB11A885B88D31A5D
:104C200018447047700200203C0300202DE9F84F23
:104C30000E46002942D0DFF890A09AF8003003F029
:104C4000FF091BB34FF000091E4F8046CB463C685E
:104C500024B325886388ED1AB54228BF354604F190
:104C6000080119442A464046FEF7BCFD63882288A5
:104C70002B449BB29A42A944A6EB0506A844638044
:104C800016D91EB19AF80030002BE0D14846BDE895
:104C9000F88F0588002DDDD1FFF758FF0220FDF7C2
:104CA00085F9044638600028F3D14846BDE8F88FFE
:104CB0002046FFF74BFFC7F800B0E2E70846BDE823
:104CC000F88F00BF700200201C0100200B4B1B78E6
:104CD0009BB110B50A4C206848B1FFF737FF00239D
:104CE00002202360FDF762F930B1FFF72FFF0220A9
:104CF000FDF75CF90028F8D110BD70471C010020B9
:104D0000700200202DE9F04FDFF8F89083B0012207
:104D100089F80020019169B3DFF8EC80364F019EDD
:104D20008346D8F80000B0B3344D4488C4F1400144
:104D3000B14228BF314604EB010E00221FFA8EFE5D
:104D40002A70761AA0F802E000F1080251B1013C85
:104D5000224459441BF8014B02F8014F8B45F9D10D
:104D6000B0F802E0BEF13F0F0BD8254A05211170C3
:104D7000002ED6D10198002389F8003003B0BDE899
:104D8000F08F4022028001460320FDF78BF90022BC
:104D9000C8F80020E9E73A782AB3184D4AF2F92416
:104DA0004FF0010A07E0013C16D02A78A2B900F0C2
:104DB000ADF83A78BAB10320FDF716F90728F2D812
:104DC00089F800A0FFF7A2FEC8F800000028ACD1C7
:104DD0000C4B013C1870E8D101234FF0FF302B70D1
:104DE00003B0BDE8F08F00234FF0FF3089F80030AA
:104DF00003B0BDE8F08F00BF1C0100206C02002052
:104E000065020020660200206802002000B583B021
:104E100002AB012103F8010D1846FFF773FF03B041
:104E20005DF804FB38B50E4D0E4C28680123237045
:104E300028B1408800232370C0F1400038BD0A4BE0
:104E40001B7813B90020207038BD0320FDF7CCF883
:104E50000728F7D8FFF75AFE28600028E9D1F1E7C4
:104E600068020020660200201C010020F8B5114BEA
:104E70001B788BB1104E114D346801272F7064B12F
:104E80000F4A638800271770214623800320FDF70F
:104E900009F9376000232B70F8BDFFF737FE084B88
:104EA00028B1014603201C70FDF7FCF8F2E71F70E3
:104EB000F0E700BF1C01002068020020660200200D
:104EC0006502002038B50E4B1B7873B90D4C216874
:104ED00061B103F0FF054B880B800320FDF7E2F87A
:104EE000256038BD084B01221A7038BDFFF70EFE51
:104EF0000028F7D00146BDE838400320FDF7D2B8BE
:104F000066020020680200206502002038B5224CAD
:104F1000237803B138BD01232370FFF779FE70BBFE
:104F2000FFF72EFA40BB00F041F810BBFFF7FEFC84
:104F3000E0B900232370EFF30583002BEAD1EFF3F0
:104F4000108172B6154B1868E0B1154C2278CAB9B9
:104F500045691D6001232370C5B1AA6101B962B61C
:104F600000254577836898472570D3E7FEF784F9D5
:104F7000DFE700F019F8D9E7FBF7E0FCD3E7FFF72C
:104F8000C3FDCDE70029C5D162B638BD054B1D6014
:104F90000029E5D1E3E700BF750200203C010020B5
:104FA0004001002038010020704700BF054A064B31
:104FB00010781B78C0B2DBB2984238BF4030C01ABC
:104FC000704700BFE80200207D020020F0B4384B9B
:104FD0001A7912F0300F2CD072B6997D01F0FF02D1
:104FE00000293DD062B6334F334938780D78334EBF
:104FF0001C46C0B2EDB2431C402BE17928BF002310
:10500000AB4202F1FF32C9B21CBFF154184612F094
:10501000FF02F0D12A4B1B68C2B23A704BB1A842D2
:1050200036BFC5F14005401B40192728C4BF0122E7
:105030001A701F49CA78D2B2150616D452060DD579
:105040001B4B1B795B0609D51E4B1F491B680022B1
:105050000A7003B11A70164B3C22DA70F0BC70472C
:105060004022D9795A7462B6E3E70B791C06E5D57C
:10507000164B174E1C783378E4B2DBB29C420ED04C
:10508000144D01E0A3420AD00133282B28BF00238E
:105090000879E85CC0B2C871087D0728F2D9DBB294
:1050A000034933700B79180644BF7C23CB70C5E7E6
:1050B00000B00640E80200207D020020A802002087
:1050C00078020020EC0200207C020020F002002088
:1050D000E90200208002002081F0004102E000BFD0
:1050E00083F0004330B54FEA41044FEA430594EAA8
:1050F000050F08BF90EA020F1FBF54EA000C55EAE3
:10510000020C7FEA645C7FEA655C00F0E2804FEAB3
:105110005454D4EB5555B8BF6D420CDD2C4480EA95
:10512000020281EA030382EA000083EA010180EAC5
:10513000020281EA0303362D88BF30BD11F0004F13
:105140004FEA01314FF4801C4CEA113102D0404249
:1051500061EB410113F0004F4FEA03334CEA133384
:1051600002D0524263EB430394EA050F00F0A7809C
:10517000A4F10104D5F1200E0DDB02FA0EFC22FA97
:1051800005F2801841F1000103FA0EF2801843FA8B
:1051900005F359410EE0A5F120050EF1200E012A7C
:1051A00003FA0EFC28BF4CF0020C43FA05F3C018BA
:1051B00051EBE37101F0004507D54FF0000EDCF133
:1051C000000C7EEB00006EEB0101B1F5801F1BD3DC
:1051D000B1F5001F0CD349085FEA30004FEA3C0CE0
:1051E00004F101044FEA445212F5800F80F09A80D6
:1051F000BCF1004F08BF5FEA500C50F1000041EBDA
:10520000045141EA050130BD5FEA4C0C404141EBDD
:10521000010111F4801FA4F10104E9D191F0000F04
:1052200004BF01460020B1FA81F308BF2033A3F187
:105230000B03B3F120020CDA0C3208DD02F1140C7E
:10524000C2F10C0201FA0CF021FA02F10CE002F1B9
:105250001402D8BFC2F1200C01FA02F120FA0CFCB2
:10526000DCBF41EA0C019040E41AA2BF01EB0451FB
:10527000294330BD6FEA04041F3C1CDA0C340EDCF9
:1052800004F11404C4F1200220FA04F001FA02F33C
:1052900040EA030021FA04F345EA030130BDC4F1FA
:1052A0000C04C4F1200220FA02F001FA04F340EAEF
:1052B0000300294630BD21FA04F0294630BD94F0A0
:1052C000000F83F4801306BF81F480110134013D87
:1052D0004EE77FEA645C18BF7FEA655C29D094EAF8
:1052E000050F08BF90EA020F05D054EA000C04BF76
:1052F0001946104630BD91EA030F1EBF0021002061
:1053000030BD5FEA545C05D14000494128BF41F0FF
:10531000004130BD14F580043CBF01F5801130BD63
:1053200001F0004545F0FE4141F470014FF00000EE
:1053300030BD7FEA645C1ABF194610467FEA655C9F
:105340001CBF0B46024650EA013406BF52EA033541
:1053500091EA030F41F4002130BD00BF90F0000F2F
:1053600004BF0021704730B54FF4806404F132046B
:105370004FF000054FF0000150E700BF90F0000F24
:1053800004BF0021704730B54FF4806404F132044B
:1053900010F0004548BF40424FF000013EE700BF1B
:1053A00042004FEAE2014FEA31014FEA02701FBFAB
:1053B00012F07F4393F07F4F81F06051704792F07D
:1053C000000F14BF93F07F4F704730B54FF46074F7
:1053D00001F0004521F0004120E700BF50EA010242
:1053E00008BF704730B54FF000050AE050EA0102EF
:1053F00008BF704730B511F0004502D5404261EB5F
:1054000041014FF4806404F132045FEA915C3FF49F
:10541000DCAE4FF003025FEADC0C18BF03325FEA38
:10542000DC0C18BF033202EBDC02C2F1200300FAED
:1054300003FC20FA02F001FA03FE40EA0E0021FA12
:1054400002F11444C1E600BF70B54FF0FF0C4CF4FC
:10545000E06C1CEA11541DBF1CEA135594EA0C0FB2
:1054600095EA0C0F00F0DEF82C4481EA030621EAED
:105470004C5123EA4C5350EA013518BF52EA033528
:1054800041F4801143F4801338D0A0FB02CE4FF0DA
:105490000005E1FB02E506F00042E0FB03E54FF00A
:1054A0000006E1FB03569CF0000F18BF4EF0010E02
:1054B000A4F1FF04B6F5007F64F5407404D25FEAFE
:1054C0004E0E6D4146EB060642EAC62141EA5551B1
:1054D0004FEAC52040EA5E504FEACE2EB4F1FD0CF3
:1054E00088BFBCF5E06F1ED8BEF1004F08BF5FEA71
:1054F000500E50F1000041EB045170BD06F0004623
:1055000046EA010140EA020081EA0301B4EB5C04CF
:10551000C2BFD4EB0C0541EA045170BD41F48011C7
:105520004FF0000E013C00F3AB8014F1360FDEBFEC
:10553000002001F0004170BDC4F10004203C35DAC8
:105540000C341BDC04F11404C4F1200500FA05F34B
:1055500020FA04F001FA05F240EA020001F00042EC
:1055600021F0004110EBD37021FA04F642EB060162
:105570005EEA430E08BF20EAD37070BDC4F10C048C
:10558000C4F1200500FA04F320FA05F001FA04F250
:1055900040EA020001F0004110EBD37041F100013C
:1055A0005EEA430E08BF20EAD37070BDC4F1200547
:1055B00000FA05F24EEA020E20FA04F301FA05F2AF
:1055C00043EA020321FA04F001F0004121FA04F257
:1055D00020EA020000EBD3705EEA430E08BF20EA27
:1055E000D37070BD94F0000F0FD101F00046400061
:1055F00041EB010111F4801F08BF013CF7D041EAE3
:10560000060195F0000F18BF704703F000465200E6
:1056100043EB030313F4801F08BF013DF7D043EAB7
:105620000603704794EA0C0F0CEA135518BF95EA6D
:105630000C0F0CD050EA410618BF52EA4306D1D1F4
:1056400081EA030101F000414FF0000070BD50EA13
:10565000410606BF1046194652EA430619D094EA9D
:105660000C0F02D150EA013613D195EA0C0F05D187
:1056700052EA03361CBF104619460AD181EA0301DB
:1056800001F0004141F0FE4141F470014FF0000093
:1056900070BD41F0FE4141F4780170BD70B54FF02E
:1056A000FF0C4CF4E06C1CEA11541DBF1CEA1355AE
:1056B00094EA0C0F95EA0C0F00F0A7F8A4EB050490
:1056C00081EA030E52EA03354FEA013100F0888087
:1056D0004FEA03334FF0805545EA131343EA126350
:1056E0004FEA022245EA111545EA10654FEA002605
:1056F0000EF000419D4208BF964244F1FD0404F5BE
:10570000407402D25B084FEA3202B61A65EB030519
:105710005B084FEA32024FF480104FF4002CB6EBD6
:10572000020E75EB030E22BFB61A754640EA0C0056
:105730005B084FEA3202B6EB020E75EB030E22BF96
:10574000B61A754640EA5C005B084FEA3202B6EBD7
:10575000020E75EB030E22BFB61A754640EA9C0096
:105760005B084FEA3202B6EB020E75EB030E22BF66
:10577000B61A754640EADC0055EA060E18D04FEA24
:10578000051545EA16754FEA06164FEAC30343EAC4
:1057900052734FEAC2025FEA1C1CC0D111F4801F91
:1057A0000BD141EA00014FF000004FF0004CB6E78A
:1057B00011F4801F04BF01430020B4F1FD0C88BF29
:1057C000BCF5E06F3FF6AFAEB5EB030C04BFB6EB34
:1057D000020C5FEA500C50F1000041EB045170BD27
:1057E0000EF0004E4EEA113114EB5C04C2BFD4EB54
:1057F0000C0541EA045170BD41F480114FF0000ED8
:10580000013C90E645EA060E8DE60CEA135594EA53
:105810000C0F08BF95EA0C0F3FF43BAF94EA0C0F56
:105820000AD150EA01347FF434AF95EA0C0F7FF4CB
:1058300025AF104619462CE795EA0C0F06D152EA1F
:1058400003353FF4FDAE1046194622E750EA410603
:1058500018BF52EA43067FF4C5AE50EA41047FF414
:105860000DAF52EA43057FF4EBAE12E74FF0FF3C79
:1058700006E000BF4FF0010C02E000BF4FF0010C4A
:105880004DF804CD4FEA410C7FEA6C5C4FEA430CC3
:1058900018BF7FEA6C5C1BD001B050EA410C0CBF12
:1058A00052EA430C91EA030F02BF90EA020F002074
:1058B000704710F1000F91EA030F58BF994208BFDB
:1058C00090422CBFD8176FEAE37040F00100704798
:1058D0004FEA410C7FEA6C5C02D150EA013C07D1EF
:1058E0004FEA430C7FEA6C5CD6D152EA033CD3D03A
:1058F0005DF8040B704700BF8446104662468C4634
:105900001946634600E000BF01B5FFF7B7FF002866
:1059100048BF10F1000F01BD4DF808EDFFF7F4FF8F
:105920000CBF012000205DF808FB00BF4DF808ED1A
:10593000FFF7EAFF34BF012000205DF808FB00BF3D
:105940004DF808EDFFF7E0FF94BF012000205DF85F
:1059500008FB00BF4DF808EDFFF7CEFF94BF012014
:1059600000205DF808FB00BF4DF808EDFFF7C4FF0D
:1059700034BF012000205DF808FB00BF4FEA410C56
:105980007FEA6C5C02D150EA013C0AD14FEA430C39
:105990007FEA6C5C02D152EA033C02D14FF0000076
:1059A00070474FF0010070470B460146184600F063
:1059B00031B800BF10B502FB01F100F06FF80446EA
:1059C000D8B150F8042C22F00302043A242A18D843
:1059D000132A14D900231B2A0360436016D9242AF2
:1059E0008360C36011BF00F110020361436100F1E5
:1059F00018020023136053609360204610BD0246D6
:105A0000F7E7002100F07CFB204610BD00F1080202
:105A1000EFE700BF13460A460146022002F056BADD
:105A2000014B1868704700BF609FFF1F70B50F4E95
:105A30000F4D761BB61018BF002405D0013455F861
:105A4000043B9847A642F9D10A4E0B4D761B04F051
:105A5000A7FDB61018BF002406D0013455F8043B4A
:105A60009847A642F9D170BD70BD00BFACA500003B
:105A7000ACA50000C0A50000ACA50000024B01468B
:105A8000186800F00BB800BF609FFF1F024B014673
:105A9000186803F09FBA00BF609FFF1F2DE9F04F09
:105AA00001F10B05162D83B0064640F29F8035F0BC
:105AB000070500F1BF80A94200F2BC8000F06EFB38
:105AC000B5F5FC7FC0F09C826B0A00F0BA80042B15
:105AD00000F28381A80900F1390E4FEA4E033830F5
:105AE000C44F07EB8303A3F108015C68A14207D10F
:105AF000ACE0002A80F2AC80E468A14200F0A6800D
:105B0000636823F003035A1B0F2AF2DDB9493C698D
:105B100001F1080E744500F0B381636823F00303BC
:105B20005A1B0F2A00F39981002AC1F814E0C1F82A
:105B300010E080F29E80B3F5007F80F06781DB0883
:105B400003F1010C01229B1002FA03F34A6851F899
:105B50003C80C4F8088001EBCC091A43A9F1080382
:105B6000E3604A6041F83C40C8F80C4083100124CF
:105B70009C40944200F28A80144206D120F0030037
:105B80006400144200F10400FAD007EBC009CC46CF
:105B90008046DCF80C108C4507D173E1002A80F2B6
:105BA0008181C9688C4500F06D814B6823F0030347
:105BB0005A1B0F2AF2DD0C46D1F80CC054F8088F9E
:105BC0004B1945F001054D6042F00101C8F80CC0C9
:105BD0003046CCF808807B613B61C3F80CE0C3F829
:105BE00008E059609A5000F0DBFA1FE0102921D834
:105BF00000F0D4FA1025062302207E4F07EB830322
:105C0000A3F108025C68944200F045816368E16892
:105C1000A56823F00303234430465A68E96042F044
:105C200001028D605A6000F0BBFA0834204603B0D0
:105C3000BDE8F08F00240C232046336003B0BDE89C
:105C4000F08F80234FF0400E3F2049E770465DE71C
:105C50002344E1685A68A56842F00102E9603046D1
:105C60008D605A6000F09CFA0834204603B0BDE80D
:105C7000F08F234430465A6842F001025A6000F027
:105C80008FFA0834204603B0BDE8F08FBC68636823
:105C900023F00308A84504D3C5EB08030F2B00F33A
:105CA0008C80554BDFF860911A68D9F800300133C9
:105CB0002A4404EB080A00F0608102F580520F329A
:105CC00022F47F6222F00F0211463046019200F06A
:105CD00059FCB0F1FF3F8346019A00F0588182459C
:105CE00000F2FC80454B1968DA451144196000F058
:105CF0005381D9F80000DFF810E101301BBFCAEB77
:105D00000B0A5144CEF800B019601BF0070100F0F7
:105D10001781C1F10800C1F58051834408315A440C
:105D2000C2F30B02C2EB010949463046019300F071
:105D300029FC431C019B00F03F81CBEB00024A444D
:105D400042F001021968C7F808B04944BC42CBF8D8
:105D500004201960DFF8A49016D0B8F10F0F40F2BC
:105D6000FD806268A8F10C0323F00703E01802F03D
:105D700001024FF0050E1A430F2B6260C0F804E0D9
:105D8000C0F808E000F21C811D4BBC681A68914203
:105D900088BF19601B4B1A689142626888BF1960FE
:105DA00022F003029542A2EB050301D80F2B04DC7D
:105DB000304600F0F5F9002438E7621943F001039A
:105DC00045F0010565603046BA60536000F0E8F9BF
:105DD0000834204603B0BDE8F08F142B71D9542B42
:105DE00000F2A480280B00F16F0E4FEA4E036E30D4
:105DF00076E600BFD0A0FF1FFC02002000030020B9
:105E0000F8020020F4020020DCA4FF1F5A0A042A32
:105E10005ED9142A00F2B38002F15C0149005B32C2
:105E200007EB810C57F82110DFF8DC81ACF1080C8E
:105E30008C4500F088804A6822F00302934202D227
:105E400089688C45F7D1D1F80CC07A68C4F80CC0C9
:105E5000A160CCF80840CC6088E6631942F00107E5
:105E600045F00105656030464B610B61C3F80CE0FD
:105E7000C3F808E05F609A50083400F091F9D5E665
:105E80004A6873E608F1010818F0030F0CF1080CDA
:105E90007FF47FAE30E0DC68A34208BF02303FF4FD
:105EA00035AEB3E60B440C465A68C96854F8085F2F
:105EB00042F001025A603046E9608D6000F070F9EE
:105EC000B4E603F15C0E03F15B004FEA4E0307E614
:105ED0009A0902F1390149003832A1E7BC424A4B24
:105EE0003FF400AF9C68626822F003025AE759F859
:105EF0000839994540F0828010F0030F00F1FF301F
:105F0000F5D17B6823EA04037B6064009C423FF682
:105F1000BDAE002C3FF4BAAE1C4240467FF435AE15
:105F200064001C4200F10400FAD02EE6B3F5AA7F0B
:105F300018D8E80B00F1780E4FEA4E037730CFE522
:105F40004FF48051EBE60121D8F80430921001FAA9
:105F500002F21A43C8F80420614677E70123CBF820
:105F6000043025E740F25452934220D8A80C00F1A7
:105F70007D0E4FEA4E037C30B2E51032A4E6542A7F
:105F800026D81A0B02F16F0149006E3248E7BC684F
:105F9000626822F0030205E7CAF30B0000287FF4D1
:105FA000A8AE4244BB6842F001025A60ECE6FE2310
:105FB0004FF07F0E7E2093E501224FF00009C1E6ED
:105FC00004F10801304603F005F8D9F80010DBE6CB
:105FD000B2F5AA7F05D8DA0B02F1780149007732D1
:105FE0001EE740F254518A4205D89A0C02F17D0115
:105FF00049007C3214E7FE217E2211E77B6884E7AA
:10600000E808431C5B00F8E5D0A0FF1F82B049B14F
:106010005AB16BB113780B601278101C18BF0120B5
:1060200002B0704701A9002AF3D1104602B07047B0
:106030006FF00100F4E700BF8842F0B50DD98B186E
:1060400098420AD28118002A51D09A1A13F8014DA9
:1060500001F8014D9342F9D1F0BD0F2A48D941EA28
:1060600000039B0746D100F1100401F1100315460F
:1060700053F8106C44F8106C53F80C6C44F80C6C2A
:1060800053F8086C44F8086C103D53F8046C44F85D
:10609000046C0F2D03F1100304F11004E8D8A2F1F1
:1060A000100323F00F0302F00F0E1033BEF1030FA5
:1060B0001944034421D91E1F0D467446043C55F86B
:1060C000047B46F8047F032CF8D8AEF1040424F0D6
:1060D000030404342344214402F0030262B1013B6F
:1060E0000A4411F8014B03F8014F8A42F9D1F0BD7F
:1060F0000346F3E70346F2E7F0BD7246EEE700BF62
:1061000070B4840746D0541E002A41D0CDB2034655
:1061100002E0621EE4B3144603F8015B9A07F8D16B
:10612000032C2ED9CDB245EA05250F2C45EA0545AD
:1061300019D903F110022646103E0F2E42F8105CCA
:1061400042F80C5C42F8085C42F8045C02F1100270
:10615000F2D8A4F1100222F00F0204F00F04103262
:10616000032C13440DD91E462246043A032A46F84E
:10617000045BFAD8221F22F003020432134404F015
:1061800003042CB1C9B21C4403F8011BA342FBD188
:1061900070BC704714460346C2E700BF704700BF9B
:1061A000704700BF2DE9F04F174683B0002900F07B
:1061B000C1800E46814607F10B05FFF7EFFF56F849
:1061C00004EC162D2EF00304A6F1080840D8102286
:1061D0001546AF4241D8944275DAC94B996808EB2D
:1061E00004008842416800F0D98021F00103034493
:1061F0005B68DB077DD51EF0010F35D03946484678
:10620000FFF74CFC0746E0B156F8043C23F00103CD
:106210004344A0F108029A4200F04481221F242A3C
:1062200000F23181132A00F20481034632461168DC
:1062300019605168596092689A603146484602F088
:10624000C9FE4846FFF7ACFF384603B0BDE8F08F03
:1062500025F00705002D2A46BBDA0C230020C9F8DB
:10626000003003B0BDE8F08F56F8083CC3EB080AD5
:10627000DAF8043023F0030C04EB0C039342BDDB8B
:106280005746DAF80C1057F8080F221F242AC1606D
:10629000886000F21781132A40F212813168CAF82F
:1062A00008107168CAF80C101B2A00F22B810836FE
:1062B0000AF110023168116071685160B168916033
:1062C0003E461C46D046631B0F2B1DD8D8F8043021
:1062D00003F0010323434444C8F80430636843F0E7
:1062E000010363604846FFF75BFF304603B0BDE83B
:1062F000F08F21F003012144914221DBC3688268C1
:106300000C46D3609A60DEE7D8F8042008EB05015C
:1063100002F00102154343F001020B44C8F8045097
:106320004A605A6842F0010208315A60484602F059
:1063300051FED7E7114603B0BDE8F04FFFF7AEBB03
:106340001EF0010F7FF45AAF56F8083CC3EB080A61
:10635000DAF8043023F0030C01EB0C0E96458BDBCE
:10636000C36882685746D3609A6057F8081FDAF806
:106370000C30CB60221F242A996000F29980132AE6
:1063800062D93368CAF808307368CAF80C301B2A1F
:1063900000F2A08008360AF1100356E021F0030B4A
:1063A000A34405F11000834559DA1EF0010F7FF474
:1063B00025AF56F8081CC1EB080ADAF8041021F0E2
:1063C000030CE34458453FF757AF5746DAF80C1033
:1063D00057F8080F221F242AC160886000F2B48099
:1063E000132A40F2A5803168CAF808107168CAF80B
:1063F0000C101B2A00F2AF8008360AF11002316837
:10640000116071685160B16891600AEB0501C5EBDC
:106410000B0242F0010299604A60DAF8043003F09E
:1064200001031D434846CAF80450FFF7B9FE384639
:106430005CE733680360736843601B2A27D800F168
:10644000080306F10802F2E63B4632681A607268F9
:106450005A60B2689A603E467446D04633E708EB0D
:106460000501C5EB0B0B4BF0010299604A6056F831
:10647000043C03F001031D43484646F8045CFFF763
:106480008FFE304632E73146FFF7D6FDD5E6B368DA
:106490008360F368C360242A28D000F1100306F15A
:1064A0001002C4E650F8043C23F003031C440AE73E
:1064B000314638467446D046FFF7BEFD3E4602E7F9
:1064C0003A46F7E6314638461C46D046FFF7B4FD5B
:1064D0003E46F8E6B368CAF81030F368CAF81430DC
:1064E000242A1BD010360AF11803AEE73369036182
:1064F0007369436106F1180200F1180397E600BFC3
:10650000D0A0FF1FB168CAF81010F168CAF81410C3
:10651000242A0FD010360AF11802CBE63369CAF8E4
:1065200018307369CAF81C3018360AF120038CE75A
:106530003A4664E73269CAF818207269CAF81C2022
:1065400018360AF12002B5E6314638460193FFF7C6
:1065500073FD019B59E7B168CAF81010F168CAF8D9
:106560001410242A03D010360AF1180247E73269C2
:10657000CAF818207269CAF81C2018360AF12002DD
:106580003DE700BF38B5074C0023054608462360A9
:10659000FDF7F2F9431C00D038BD2368002BFBD077
:1065A0002B6038BD580300200EB4F0B59CB021AB71
:1065B0000F4953F8042B019305466FF00044086817
:1065C00002954FF402774FF6FF7602A90695ADF8D3
:1065D000147004940794ADF8166000F07FF8029BE5
:1065E00000221A701CB0BDE8F04003B0704700BF35
:1065F000609FFF1FFFFFFFFFFFFFFFFFFFFFFFFF8A
:1066000090F800F06DE9024520F007016FF0000CF2
:1066100010F0070491F820F040F049804FF000049A
:106620006FF00700D1E9002391F840F000F1080075
:1066300082FA4CF2A4FA8CF283FA4CF3A2FA8CF3AD
:106640004BBBD1E9022382FA4CF200F10800A4FA14
:106650008CF283FA4CF3A2FA8CF3E3B9D1E9042368
:1066600082FA4CF200F10800A4FA8CF283FA4CF39F
:10667000A2FA8CF37BB9D1E9062301F1200182FA59
:106680004CF200F10800A4FA8CF283FA4CF3A2FA5F
:106690008CF3002BC6D0002A04BF04301A4612BA6D
:1066A000B2FA82F2FDE8024500EBD2007047D1E970
:1066B000002304F00305C4F100004FEAC50514F0FF
:1066C000040F91F840F00CFA05F562EA05021CBFD0
:1066D00063EA050362464FF00004A9E72DE9F04F95
:1066E000C1B00C46099115460E930A9002F05AFD6E
:1066F000036817931846FFF783FFA38916901E06B9
:1067000003D52369002B01F01A8100231A46129346
:106710002593249319930B93DFF864A4149230AB60
:10672000239399461592A84698F800304446EBB159
:10673000252B02D11AE0252B03D014F8013F002BA2
:10674000F9D1C8EB04058DB1249B259AC9F80080C6
:1067500001332A44072BC9F804502592249300F3EF
:10676000A68009F108090B9B2B440B932378002B7F
:1067700000F0A68000231A468DF86F3019460C935E
:1067800007934FF0FF3B637804F101085D4608F181
:106790000108A3F12000582800F22584DFE810F05A
:1067A00088032304230490032304230423042304E1
:1067B000230423049703A50323045D00E2002304BC
:1067C000FE000501050105010501050105010501A1
:1067D00005010501230423042304230423042304C3
:1067E00023042304230423041501810223048102CA
:1067F0002304230423042304C60223042304CD0218
:1068000023042304230423042304F702230423047E
:10681000250323042304230423042304230423043F
:106820002304230423046603790381028102810285
:106830008103790323042304D1032304DB03A3008E
:106840006400EE032304F5032304AA0323042304B2
:10685000BC030C980E9340420C90079B43F004033A
:10686000079398F8003092E70E98AB460021046831
:106870008DF86F10071D0798302378228B458DF80F
:1068800070304FF000058DF8712040F00203C0F227
:10689000C78320F0800343F00203079354EA050303
:1068A0000E9700F093830F461192B348CEE223AACD
:1068B00009990A9802F0E2FF48B90DF1C00952E7C0
:1068C000259B23B10A98099923AA02F0D7FF099BB7
:1068D0009B8913F0400F0B9B18BF4FF0FF331846F6
:1068E00041B0BDE8F08F1193AB46002A41F03382EE
:1068F000079A12F0200300F02E820E9F073727F030
:106900000703002703F10801BB450E91D3E90045B9
:106910008DF86F70C0F2798722F08003079354EAF4
:10692000050300F0758330AEE20842EA4572E908DB
:1069300004F007030D461446303354EA050206F806
:10694000013DF1D1079AD10740F18480302B00F04E
:1069500081803022731E06F8012C30AAD21A0D92C3
:106960001E467AE098F800302A2B08F1010401F065
:10697000B981A3F13000092898BF002501F26C818C
:1069800014F8013B05EB850500EB4505A3F130004C
:106990000928F5D945EAE575A046FAE6079B43F0D4
:1069A0008003079398F80030F1E6A3F1300000234C
:1069B0001C4618F8013B04EB840400EB4404A3F1EB
:1069C00030000928F5D90C94E3E61193AB46002A70
:1069D00041F0AB81079B43F010030793079B980698
:1069E00040F130850E9F073727F00707D7E90023CE
:1069F00007F108010E9114461D46002A73F10003A9
:106A0000C0F25B85BBF1000F9DF86F70C0F2388556
:106A1000079B23F08003079354EA050300F0DB8112
:106A2000002D08BF0A2CC0F0DB8130AE204629467D
:106A30000A22002302F0FAFF303206F8012D204628
:106A4000294600230A2202F0F1FF04460D4654EACB
:106A50000503EBD130AB9B1B0D930D9B5B45B8BF82
:106A60005B4608930023139317B1089B01330893E7
:106A7000079B13F002030F9302D0089B0233089385
:106A8000079B13F08403109340F0D7820C9B089A65
:106A90009D1A002D40F3D182102D2599249A374F4D
:106AA00027DD189648461024B946099E2F460A9DB0
:106AB00004E0103F102F00F1080016DD01322F4BCB
:106AC00024921031072A259180E81800F1DD23AACD
:106AD0003146284602F0D2FE00287FF4F8AE103F7F
:106AE000102F2599249A30A8E8DC189E3D464F4681
:106AF000814601326C18072A25942492C9F8007047
:106B0000C9F8045000F328849DF86F7009F1080952
:106B100077B1249B013301340DF16F010122072B62
:106B20002594249389E8060000F3A08309F108095D
:106B30000F9B6BB1249B013302341CA90222072B4B
:106B40002594249389E8060000F39C8309F1080941
:106B5000109B802B00F0D5820D9BC3EB0B07002F01
:106B600039DD074A249B0F92102F28DD22464FF073
:106B7000100B0A9D099C0AE05CA300007CA30000A6
:106B800028A30000103F102F09F1080916DD01337A
:106B90001032072B2592249389E8000CF2DD23AAFA
:106BA0002146284602F06AFE00287FF490AE103F8E
:106BB000102F259A249B0DF1C009E8DC14460133FF
:106BC0000F9A24933C44072B259489E8840000F312
:106BD000418309F10809079BDA0500F13082249B03
:106BE0000D99C9F8006001330C44072B2594C9F8AE
:106BF0000410249300F3188309F10809079B59072F
:106C00003FD50C9B089A9D1A002D3ADD102D249B30
:106C1000BC4F23DD22461026DDF828B0099C04E095
:106C2000103D102D09F1080917DD0133B5492493F2
:106C30001032072B259289E84200F1DD23AA214674
:106C4000584602F01BFE00287FF441AE103D102D87
:106C5000259A249B0DF1C009E7DC144601332C442E
:106C6000072B25942493C9F80070C9F8045008DD57
:106C700023AA09990A9802F001FE00287FF427AEA2
:106C8000259C0B9B0C9A08998A42ACBF9B185B18F9
:106C90000B93002C40F0D482002324930DF1C00903
:106CA00042E51193AB46002A41F051800E9F073711
:106CB00027F0070303F108020E921A6814925B682A
:106CC0001593159B149D23F00044284621464FF050
:106CD000FF328D4BFEF752FE002840F0C28428465A
:106CE00021464FF0FF32884BFEF72AFE002840F085
:106CF000B8841498159900220023FEF717FE002887
:106D000040F04F879DF86F70804E814B079921F0BE
:106D100080010791119903224FF0000B0892472937
:106D2000D8BF1E460D92CDF84CB09DE6079B43F0B0
:106D30000803079398F8003029E51193AB46002A21
:106D400041F01180079B43F010030793079A12F05C
:106D500020037FF4D2AD079911F0100200F02C85CA
:106D60000E988DF86F30BBF1000F046800F1040736
:106D70004FF00005C0F248850A4622F080020792D3
:106D800054EA05020E9700F043811F46CBE51193AC
:106D9000AB46002A40F0E387079B43F010030793BC
:106DA000079A12F0200300F032830E9F073727F076
:106DB0000703002703F10801BB450E91D3E9004505
:106DC0008DF86F70C0F25C8322F08003079354EA61
:106DD00005037FF425AEBBF1000F00F0FE80002418
:106DE00040AE303406F8414D34E61193AB46002AEC
:106DF00040F09787079B47489D0640F197800E9F7C
:106E0000073727F00703D3E9004503F108020E9284
:106E1000079A12F0010700F0418254EA050300F0DE
:106E200005859DF844208DF871200027079A8DF87C
:106E30006F703023BB458DF8703042F00203C0F212
:106E4000B58622F0800343F00203079330AE230996
:106E500004F00F0143EA05732A091C461546435CFA
:106E600006F8013D54EA0503F1D1F3E50E991193BB
:106E70000A688DF8982000230A461F468DF86F3067
:106E8000043201230893BB4613970E920D9326AE4E
:106E9000EEE51193AB46002A3FF4A0AD8DF86F10DC
:106EA0009CE5079B43F04003079398F800306EE49D
:106EB00098F8003000297FF46AAC0122202166E4B2
:106EC000079B43F00103079398F800305FE40E9CA2
:106ED00023680C9318460028234603F10403FFF6A9
:106EE000B8AC0E9398F8003051E498F800300122C5
:106EF0002B214CE41193AB46002A3FF451AF8DF89F
:106F00006F104DE77CA30000FFFFEF7F3CA3000064
:106F100038A3000048A300001193AB46002A40F0BC
:106F20002A87079B99489D063FF569AF079BDC06BA
:106F300040F135840E9A1346043314680E930025ED
:106F400066E798F800306C2B00F0E284079840F078
:106F5000100007901BE4002A40F00987079B9B065E
:106F600040F106840E9A0B991368CD170846043237
:106F700029460E92C3E90001FFF7D6BB079B43F0F9
:106F80002003079398F8003001E40E9A11931668D5
:106F900000248DF86F40171D002E00F0CD85002DC8
:106FA000C0F218852A462146304602F009F9002829
:106FB00000F02A86831B0D93A34623EAE3730E9702
:106FC0000893CDF84CB09DF86F704DE56F48119265
:106FD000BBF1000F40F073815F464FF0000BCDF81E
:106FE00034B030AE39E51193002A40F0AC86119AE6
:106FF000002A3FF465AC002301211F4608918DF85B
:1070000098208DF86F309B4613930D9126AE2FE597
:10701000BBF1000F00F0038600270024002582E466
:107020005A480793119254EA05030E974FF0000750
:107030007FF40CAF0024002508E7259C68E5119B30
:10704000652B40F3A9801498159900220023FEF7C0
:1070500063FC002800F03581249B4D4AC9F80020CC
:10706000013301340122072B25942493C9F804200D
:1070700000F3E88309F108091D9B129A934203DB90
:10708000079BDB077FF5BAAD249B1699179AC9F8C1
:10709000002001330C44072B2594C9F804102493D5
:1070A00000F3408409F10809129B5D1E002D7FF753
:1070B000A5AD384A249B0F92102D40F3E68110268F
:1070C0000A9FDDF824B005E009F10809103D102DF4
:1070D00040F3DB8101331034072B25942493C9F846
:1070E00000A0C9F80460EFDD23AA5946384602F033
:1070F000C5FB00287FF4EBAB259C249B0DF1C00958
:10710000E4E70C9B089A9F1A002F7FF725AD214AD0
:10711000249B0F92102F2BDD4A462146B94610259D
:1071200037460A9C099E06E0A9F11009B9F1100F33
:1071300002F1080218DD01331031072B2591249349
:10714000C2F800A05560EFDD23AA3146204602F0C8
:1071500095FB00287FF4BBABA9F11009B9F1100F22
:107160002599249B30AAE6DC3E460C464F469146C4
:1071700001330F9A24933C44072B259489E884001B
:1071800000F3458209F10809E6E400BF5CA30000B2
:1071900078A3000028A30000129B249D012B40F33C
:1071A0000882013501340123072D25942495C9F85F
:1071B0000060C9F8043000F30D8209F10809169A3D
:1071C000179BC9F8003001351444072D25942495E8
:1071D000C9F8042000F30E8209F10809002314986D
:1071E00015990022FEF798FB129B002840F0C380FF
:1071F000013B013501361C44072D24952594C9F81F
:107200000060C9F8043000F3F58009F10809199A03
:10721000C9F80420013514441FAB072D259424958B
:10722000C9F800307FF7E8AC23AA09990A9802F060
:1072300025FB00287FF44BAB259C0DF1C009DDE454
:1072400023AA09990A9802F019FB00283FF424ADFB
:10725000FFF73DBB23AA09990A9802F00FFB00280B
:107260007FF435AB259C0DF1C009B4E423AA09993C
:107270000A9802F003FB00287FF429AB259C0DF14E
:10728000C00955E423AA09990A9802F0F7FA0028E0
:107290007FF41DAB259C0DF1C00959E4BBF1000F33
:1072A0008DF86F70C0F2DA8222F08003079354EAFF
:1072B00005037FF4CBADBBF1000F3FF48DAE00278B
:1072C000B8E61D9D002D40F3CC82139B129A934289
:1072D000A8BF1346002B1D460DDD249BC9F8006096
:1072E00001332C44072B2594C9F80450249300F350
:1072F000A38309F10809139B002DA8BF5B1B002B7A
:107300001D4640F3F680BA4A249B0F92102D40F39D
:10731000808222461027DDF828B0099C05E009F19B
:107320000809103D102D40F3738201331032072BF2
:1073300025922493C9F800A0C9F80470EFDD23AAB0
:107340002146584602F09AFA00287FF4C0AA259AEE
:10735000249B0DF1C009E4E723AA09990A9802F0D9
:107360008DFA00287FF4B3AA9DF86F70259C0DF16B
:10737000C009FFF7CDBB5E1E002E7FF748AF9C4BC8
:107380000F93102E2CDDCDF834801027B046DDF899
:1073900028B0099E06E0A8F11008B8F1100F09F115
:1073A00008091ADD01351034072D25942495C9F8F4
:1073B00000A0C9F80470EEDD23AA3146584602F059
:1073C0005DFA00287FF483AAA8F11008B8F1100F25
:1073D000259C249D0DF1C009E4DC4646DDF834808F
:1073E0000F9B01353444072D2594249589E84800E6
:1073F0007FF70BAF23AA09990A9802F03FFA0028F9
:107400007FF465AA259C249D0DF1C009FFE607992C
:1074100011F0100200F008810E988DF86F30BBF16A
:10742000000F046800F104074FF0000526DB0A4650
:1074300022F08002079254EA05020E971F467FF45D
:10744000EFAAC8E4079BD9062AD4079B5A0627D57A
:107450000E99B1F900400431E51722462B460E91F2
:10746000FFF7CBBA0E998DF86F30BBF1000F0C68A7
:1074700001F104074FF0000580F245820E971F4688
:1074800054EA05037FF4CCAAAAE401330F9A2493AB
:107490002C44072B259489E824007FF7ADABC3E685
:1074A0000E9A146813460433E51722460E93002AF9
:1074B0002B4673F10003BFF6A5AA64424FF02D07D7
:1074C00065EB4505BBF1000F8DF86F70FFF6A8AABC
:1074D000079B23F080030793FFF7A2BA23AA099919
:1074E0000A9802F0CBF900287FF4F1A9259C0DF150
:1074F000C009139A1D9B32441746129A934247DBE8
:10750000079AD50744D412990E44F51BCB1A9D4215
:10751000A8BF1D46002D2E460DDD249AC9F8007027
:1075200001322C44072A2594C9F80450249200F310
:10753000128309F10809002EACBF9D1B1D46002DCA
:107540007FF75CAB2A4A249B0F92102D9DDD1026FD
:107550000A9FDDF824B004E009F10809103D102D60
:1075600093DD01331034072B25942493C9F800A030
:10757000C9F80460F0DD23AA5946384602F07EF9C6
:1075800000287FF4A4A9259C249B0DF1C009E5E700
:10759000249A16981799C9F8001001320444072A52
:1075A0002594C9F80400249200F3A58209F1080982
:1075B000A9E7079BD8073FF5F4AD01350134012356
:1075C000072D25942495C9F80060C9F804307FF789
:1075D0001CAE0FE723AA09990A9802F04FF9002878
:1075E0007FF475A9259C249D0DF1C009E7E500BF36
:1075F00028A3000023AA09990A9802F03FF900285D
:107600007FF465A9259C249D0DF1C009E6E523AA18
:1076100009990A9802F032F900287FF458A9259CAC
:107620000DF1C009FFF798BA079911F040033FF434
:1076300019AF0E988DF86F200346BBF1000F03F1D0
:10764000040304884FF00005C0F2B98121F08001E5
:10765000079154EA05010E9317467FF4E1A9FFF75D
:10766000BABB149C22462046159C23462146FEF7B1
:1076700085F9002840F01583119BBBF1FF3F23F0F3
:1076800020030D9300F07682472B00F09281079B38
:1076900043F480731093159B1F1E149B0893BBBF6C
:1076A0003B4603F1004700232D230F93119B662BCC
:1076B00000F06382462B00F05E810D9B089A452BFB
:1076C00021A81EA90CBF0BF101055D460490039192
:1076D0001DA802213B460290019500910A9800F0F6
:1076E000EBFC119B672B064640F07D82079BDA0777
:1076F00040F1BF8274190898394600220023FEF732
:107700000BF9002840F0A481219B9C4206D930212E
:107710005A1C21921970219B9C42F9D89B1B1293F1
:107720000D9B472B00F08181119B652B40F36A82F2
:10773000119B662B1D9B139300F04782139A12999D
:107740008A42C0F23682079BD90700F1898222EA79
:10775000E2730D92672211920F9A002A40F05B812A
:107760000893109B079393469DF86F70FFF77CB9C1
:10777000079BDF060BD4079B5E0608D50E9A13689D
:1077800004320E92BDF82C201A80FEF7CDBF0E9A5F
:10779000136804320E920B9A1A60FEF7C5BF079B5E
:1077A0000E9A13F0400F134600F00E810433148834
:1077B0000E930025FFF72CBB079911F0400317D05B
:1077C0000E988DF86F200346BBF1000F03F1040300
:1077D00004884FF00005C0F2F58021F08001079188
:1077E00054EA05010E933FF413AC1746FFF79BB81C
:1077F0000E998DF86F30BBF1000F0C6801F1040792
:107800004FF0000580F281800E970027FFF78BB8BC
:10781000144601330F9A24932C44072B259489E8AE
:1078200024003FF75BAE09F1080962E60027BB457B
:107830008DF86F70FFF6FEAB079B23F08003079374
:10784000FFF7C6BB23AA09990A9802F017F8002887
:107850007FF43DA8259C0DF1C0090DE40E9FFFF7B4
:10786000E2BB249BB14AC9F8002001330134012254
:10787000072B25942493C9F804206FDC09F108092B
:107880002DB9129B1BB9079BDF077FF5B7A9249B76
:107890001699179AC9F8002001330C44072B259438
:1078A000C9F80410249300F3C98109F108096D4255
:1078B000002D40F3A3809E4A0F92102D40F32981A2
:1078C00022461027DDF828B0099C05E009F10809D7
:1078D000103D102D40F31C8101331032072B2592EF
:1078E0002493C9F800A0C9F80470EFDD23AA21464B
:1078F000584601F0C3FF00287EF4E9AF259A249B87
:107900000DF1C009E4E7079A92E5079AFFF735BA47
:10791000079B43F02003079308F1010898F8003013
:10792000FEF735BF23AA09990A9801F0A7FF00289E
:107930007EF4CDAF259C0DF1C009FFF7B5BB40210A
:107940000A98FEF7ABF8099A10601061002800F061
:10795000F381099A40235361FEF7D7BE23AA099900
:107960000A9801F08BFF00287EF4B1AF1D9D259C85
:107970000DF1C00984E721A81EA9049003911DA858
:1079800003210290089ACDF804B03B4600910A9872
:1079900000F092FB5D460646119B462B06EB050464
:1079A0007FF4A9AE3378302B00F06D811D9D2C44FF
:1079B000A1E6BBF1000F08BF4FF0010B67E60E9385
:1079C00017465DE50E9320E7043314680E930025F7
:1079D000FFF71EBA3046FEF713FEA34603460D908E
:1079E000FFF7EBBA23AA09990A9801F047FF00288C
:1079F0007EF46DAF259C249B0DF1C0091299C9F846
:107A0000006001330C44072B25942493C9F804101B
:107A10007FF7F2A808E42D270893109B07938DF8B1
:107A20006F704FF0000BFFF720B81D9BDD1C11DBC2
:107A30009B450FDB139381E623AA09990A9801F06D
:107A40001DFF00287EF443AF259C0DF1C00952E4D0
:107A5000234663E6119A023A1192013B002B9DF8EE
:107A600044201D93B8BF5B428DF87C20B4BF2D220B
:107A70002B22092B8DF87D2040F3FD800DF18B002A
:107A800004462C4A82FB0321DA17C2EBA10202EB67
:107A90008201A3EB410303F13001092A134604F8E4
:107AA000011DEEDC21463033DAB201F8012D8842A7
:107AB00040F23F810DF17E01234601E013F8012BD6
:107AC00001F8012B9842F9D1431C1B1B0DF17E02DA
:107AD00013441FAA9B1A129A1993012A13440D9357
:107AE00040F3F6800D9B169A134400220D931392D7
:107AF00023EAE37330E623AA09990A9801F0BEFE4F
:107B000000287EF4E4AE1D9B259C0DF1C009FAE42B
:107B1000144601330F9A24932C44072B259489E8AB
:107B200024003FF75FAF09F1080967E778A3000079
:107B300028A3000067666666062D2B4628BF06232D
:107B40000D9323EAE373B3460E97139637460893D3
:107B50008B4EFEF789BF23AA09990A9801F08EFE81
:107B600000287EF4B4AE1D9B129A259CD31A0DF109
:107B7000C009E0E44FF0060B89E521A81EA9049096
:107B800003911DA803210290089ACDF804B03B464A
:107B900000910A9800F090FA5D46064600EB0B044F
:107BA00000E72D278DF86F70FFF7AEB80793FFF74A
:107BB0004DB9169A129B1344139A0D93002A7FDD38
:107BC000672223EAE3731192C6E5002B40F3988005
:107BD000BBF1000F6BD1079AD40768D41A460D92F7
:107BE00023EAE373B8E5119B472B7FF483AD079B32
:107BF000DB073FF5D1AE219B9B1B12930D9B472BBF
:107C00003FF413AF1D9B28E725EAE5730E97089311
:107C10000D95834613909DF86F70FEF725BF079B67
:107C2000DB075F4605D540AE302306F8413DFEF741
:107C300011BFCDF834B030AEFEF70FBF23AA0999BB
:107C40000A9801F01BFE00287EF441AE1D9D259C84
:107C5000249B0DF1C0092AE6A0460025FEF799BD38
:107C6000169A139B134467220D93119223EAE37330
:107C700072E5219B52E5303330228DF87F308DF84C
:107C80007E2020AB25E70898394600220023FDF727
:107C900043FE00287FF48AAEC5F101051D952C44F2
:107CA00029E5384E384B9DF86F70FFF72FB8139BBE
:107CB000169A9D1805EB0B030D9323EAE3734BE52E
:107CC000139B0D9AC3F101031A4413460D9277E7F3
:107CD000079B13F001037FF405AF13930D9B23EA79
:107CE000E37339E50E9898F8013005680430002DEB
:107CF0000E90A046BEF64BAD4FF0FF35FEF747BDE8
:107D0000BBF1000F02D1079BD80707D5169B5D1C5E
:107D100005EB0B030D9323EAE3731DE501230D939C
:107D20001AE58DF86F10FFF765B88DF86F10FEF744
:107D300051BE0DF17E03CCE60A9A0C2313604FF07E
:107D4000FF30FEF7CDBD8DF86F10FFF750B98DF8FD
:107D50006F10FEF7ABBF8DF86F10FEF7C9BD8DF841
:107D60006F10FFF719B88DF86F10FEF7EBBF8DF8A5
:107D70006F10FFF7F3B88DF86F10FFF7D2B800BFA0
:107D800070A3000044A3000040A30000F0B5ADF5CF
:107D9000057D04AD00930F4613464FF4007403AA0B
:107DA00029460394064601F0E9FD88B104460246DF
:107DB0003946039B304600F073F8AC42039004D080
:107DC0003046214601F006F903980DF5057DF0BD1A
:107DD0004FF0FF30F9E700BF10B4044C13460A46D9
:107DE0000146206810BCFFF7D1BF00BF609FFF1F96
:107DF00070B5002A9AB005462FDB14461A464FF498
:107E0000027300910491ADF80C3011D0013C4FF693
:107E1000FF761E9B029469460594ADF80E60FEF74E
:107E20005DFC421C12DB009B00221A701AB070BD70
:107E30001E9B02944FF6FF7669460594ADF80E60DE
:107E4000FEF74CFC431C04DB1AB070BD8B232B6087
:107E5000E9E78B232B601AB070BD8B2303604FF0D2
:107E6000FF30F1E710B582B0054C0093246813464B
:107E70000A4601462046FFF7BBFF02B010BD00BF17
:107E8000609FFF1F21B1FF2A04D80A7001207047AC
:107E9000084670478A2303604FF0FF30704700BFE9
:107EA00070B50D46084C114606461A462846002372
:107EB0002360FBF7F3F9431C00D070BD2368002B4F
:107EC000FBD0336070BD00BF580300202DE9F047A0
:107ED000254C2568D5F8484106468846924699467D
:107EE000C4B360681F2817DC431C76B104EB80051F
:107EF0000122C5F888A0D4F8881182401143022ECF
:107F0000C4F88811C5F808911ED00230636044F8A7
:107F100020800020BDE8F087144B03B34FF4C870F5
:107F2000FDF7ACFD0446D0B1D5F84831002780E814
:107F30008800C5F8484138460123C4F88871C4F860
:107F40008C71002EE1D0D1E7D4F88C110A43C4F82B
:107F50008C21DAE705F5A674C5F84841C1E74FF072
:107F6000FF30BDE8F08700BF14A300007D5A000079
:107F7000024B13B1024800F005B870470000000042
:107F8000118F0000002301461A461846FFF79EBFD6
:107F900002690B69934200F38D802DE9F04F03F1E4
:107FA000FF3801F1140700F1140B57F828205BF893
:107FB00028304FEA880483B00132B3FBF2F90BEBAF
:107FC0000403009407EB040A0193B9F1000F39D0C0
:107FD0000025BC46DE462B465CF8046BDEF800202C
:107FE000B4B209FB0455360C2C0C09FB0644ADB2A7
:107FF0005B1BA6B213FA82F3C6EB124606EB2346CE
:108000009BB243EA0643E2454EF8043B4FEA14456F
:108010004FEA2643E0D2009B5BF8033093B9019C02
:10802000231F9B450CD254F8043C4BB9A4F1080320
:1080300002E01A68043B1AB99B4508F1FF38F8D3EF
:10804000C0F81080044601F013FB00282EDB09F174
:1080500001095D46002357F8041B28688AB29A1A62
:10806000090C12FA80F2C1EB104303EB224391B2E8
:1080700041EA0341BA4545F8041B4FEA2343EAD2DB
:108080005BF828200BEB880382B91A1F93450BD2AB
:1080900053F8042C42B9083B02E01A68043B1AB9B1
:1080A0009B4508F1FF38F8D3C4F81080484603B068
:1080B000BDE8F08F002070472DE9F04F016C97B0BC
:1080C0008146239C92469B4649B1426C4A600123FB
:1080D00093408B6001F0EAF80023C9F84030BBF10F
:1080E000000FD84633DB00232360A54B1A4608EA6D
:1080F0000303934214D05046594600220023FDF753
:108100000BFC054648B3229A01231360249B002BE5
:1081100000F0C5809B481860013817B0BDE8F08FAB
:10812000229A42F20F731360BAF1000F00F0A2809E
:108130009548249B002BF0D0C378002B00F0B18031
:1081400000F10803249A136017B0BDE8F08F0123F3
:108150002BF000482360C346C7E714AA15AB019271
:10816000009352465B46484601F02CFB5FEA1854E8
:10817000089040F08880149D159C2C4404F23243F2
:10818000202B40F39182C3F1400304F2124008FA1D
:1081900003F82AFA00F040EA0800FDF7DFF80123AF
:1081A000013CA1F1F87110930022784BFCF798FF85
:1081B0006DA3D3E90023FDF747F96DA3D3E90023AD
:1081C000FCF790FF064620460F46FDF7D7F86AA356
:1081D000D3E90023FDF738F902460B46304639460D
:1081E000FCF780FF06460F4601F0F8FB00220490E2
:1081F000002330463946FDF799FB002840F03082D5
:10820000049E162E00F22982614B03EBC603D3E9CC
:10821000000152465B46FDF7A7FB002800F04982AB
:10822000731E049300230C932C1B631E029300F116
:10823000328200230593049B002BC0F22382029A12
:108240000B9311461944002302910A93209B092B9A
:1082500029D8052B40F35886043B20930025209B0A
:10826000023B032B00F23586DFE813F02C032802D3
:1082700037035904444B474AC8F31300002814BF7E
:108280001846104655E7CBF3130343F07F51109582
:108290005046A4F2FF3441F44011149D84E73E4857
:1082A0003BE7C31C4EE70021C9F844104846209123
:1082B00000F0D6FF4FF0FF330693209A0D93012371
:1082C00007902192C9F840000993159B002BC0F23A
:1082D000D180049A0E2A00F3CD802D4B03EBC2030C
:1082E000D3E90034CDE90234219B002BC0F2008396
:1082F00056465F4650465946DDE902AB52465B465C
:10830000FDF7CCF901F06AFB0446FDF737F8524659
:108310005B46FDF799F80B46024639463046FCF7B6
:10832000DFFE079D04F130032B70069B012B0646F0
:108330000F4605F1010562D00022184BFDF784F8C5
:108340000022002306460F46FDF7E6FA00287ED1FC
:10835000CDF81490DDF818A0DDF81CB0DDE9028935
:1083600029E000BFAFF3008061436F63A787D23F6E
:10837000B3C8608B288AC63FFB799F501344D33F14
:108380000000F07F79A300009CA400000000F83FEB
:10839000A0A4000090A4000078A3000000002440E6
:1083A000FDF752F80022002306460F46FDF7B4FA07
:1083B000002840F0B78342464B4630463946FDF729
:1083C0006DF901F00BFB0446FCF7D8FF42464B4623
:1083D000FDF73AF802460B4630463946FCF780FE78
:1083E00004F1300E05F801EBCBEB050ED645064641
:1083F0000F464FF00002B04BD2D1DDF81490324658
:108400003B4630463946FCF76DFE06460F460246AF
:108410000B46DDE90201FDF789FA40B932463B46D9
:10842000DDE90201FDF778FA88B1E3070FD515F809
:10843000014C079A6B1E04E09A4200F02C8413F85A
:10844000014D392C03F10105F6D001341C70089957
:10845000484600F02BFF0022049B2A70229A013329
:108460001360249B002B00F0A78307981D6017B0B2
:10847000BDE8F08F099A002A00F01281209A012AA3
:1084800040F35882069B0A9A5F1EBA42C0F2978355
:10849000D71B069B002BC0F28A84059D069B059A7C
:1084A0001A440592029A01211A444846029200F0A9
:1084B00095FF064665B1029900290B4608DDA942E1
:1084C000059AA8BF2B46D21AED1ACB1A0592029331
:1084D0000A9B002B40F3FC82099A002A00F00182DB
:1084E000002F00F0FE8131463A46484601F018F868
:1084F000DDF82080014642460646484600F078FFF7
:1085000041460446484600F0D1FE0A9BDB1B0A9315
:1085100040F0E6810121484600F060FF0B9B804659
:10852000002B00F0198201461A46484600F0F8FF79
:10853000209B012B804640F3F8820027D8F81030AA
:1085400008EB8303186900F0FBFEC0F12000029ADB
:10855000104410F01F0000F0F681C0F12003042B3E
:1085600040F3CA84059BC0F11C00034405931346E5
:10857000034405440293059B002B05DD21461A4662
:10858000484601F01DF80446029B002B05DD4146DC
:108590001A46484601F014F880460C9B002B40F028
:1085A0007C82069B002B40F39582099B002B40F0B8
:1085B000F581DDF81CB0069F5D4602E000F080FE0C
:1085C000044641462046FFF7E3FC00F1300A05F877
:1085D00001ABCBEB0503BB424FF00A024FF00003A7
:1085E00021464846EADB079B069A012AACBF9B1846
:1085F00001331D464FF0000B21460122484600F092
:10860000DFFF4146089001F033F8002840F30D8366
:1086100015F8012C07996B1E04E08B4200F078825C
:1086200013F8012D392A03F10105F6D001321A7031
:108630004146484600F03AFE002E3FF408AFBBF139
:10864000000F05D0B34503D05946484600F02EFE32
:108650003146484600F02AFEF9E601230C93E3E593
:10866000DDF810804046FCF789FE02460B46304696
:108670003946FDF751F900287FF4C2AD08F1FF3308
:108680000493BDE5059A049BD21A5B420A9300232A
:1086900005920B93DAE55B42059300230293CAE54A
:1086A0000A9F059D099E05E7C3F120080AFA08F014
:1086B00073E50C90B8E500BF000024400023099347
:1086C000049B219A13440D930133002B069340F32E
:1086D0008382069C26460021172EC9F844100BD928
:1086E000012204235B0003F11400B042114602F1A1
:1086F0000102F7D9C9F84410484600F0B1FD0E2C2C
:108700000790C9F840003FF6E0AD002D3FF4DDAD25
:1087100004995746D8460029CDE90E7840F3928255
:10872000914B01F00F020E1103EBC203F006D3E9E7
:10873000004540F14C828D4B50465946D3E9082301
:10874000FCF7ACFF06F00F0682468B464FF003089D
:1087500086B1864FF10709D520462946D7E900237F
:10876000FCF772FE08F1010804460D46761007F189
:108770000807EFD122462B4650465946FCF78EFF9C
:1087800006460F460C9B43B10022794B30463946D2
:10879000FDF7CCF8002840F020834046FCF7EEFDC2
:1087A00032463B46FCF750FE724B0022FCF79AFC27
:1087B000069B0446A1F15075002B00F0DF81049B5D
:1087C000DDF818801193099B002B00F09782664B0F
:1087D000694903EBC80353E902230020FCF75EFF5D
:1087E00022462B46FCF77CFC82468B4630463946B7
:1087F00001F0F4F80446FCF7C1FD02460B46304692
:108800003946FCF76DFC3034079DE4B206460F464E
:108810002C7002460B46504659460135FDF7A4F828
:1088200000284CD132463B4600205149FCF758FC09
:1088300002460B4650465946FDF796F8002840F090
:108840000D83B8F1010F40F3B381079B98440DE00D
:1088500000204749FCF744FC52465B46FDF766F8AA
:10886000002840F0FB82454500F0A2815046594661
:108870000022424BFCF7E8FD0022404B82468B462B
:1088800030463946FCF7E0FD0F46064601F0A6F8F3
:108890000446FCF773FD02460B4630463946FCF7AA
:1088A0001FFC3034E4B252465B4605F8014B0646E5
:1088B0000F46FDF73BF832463B460028C8D0119BD7
:1088C0000493C4E500230993219B002B40F3898185
:1088D0001E461C460D930693FDE601230993F3E71C
:1088E00008940A9A0899484600F01AFE044611E6D0
:1088F000069B002B3FF7FCAC40F0DA820022204BB5
:10890000DDE90201FCF7A0FD52465B46FDF722F8C7
:10891000DDF818804646002800F0F280219B079D74
:10892000DB4304934146484600F0C0FC002E3FF470
:108930008EAD8DE6109A002A00F0418203F2334397
:108940000A9F059DABE51C20059B03440593029BF4
:108950000344054402930EE6209B012B40F38282E0
:108960000B9F0120F3E500BFA0A4000078A5000044
:108970000000F03F00001C400000E03F00002440E9
:1089800000001440314600230A22484600F098FCBB
:108990000D9B002B064640F397820693002D05DDC4
:1089A00031462A46484600F00BFE0646002F40F0AE
:1089B0007C810596069B079ADDF814B0013BD3181D
:1089C00008930AF0010309931746C2465146204610
:1089D000FFF7DEFA31460546204600F049FE5A46CA
:1089E00002905146484600F063FEC268804605F199
:1089F0003003002A49D101462046069300F038FE94
:108A000041460590484600F051FC059A069B2AB95C
:108A1000209919B90999002900F036820299002994
:108A2000C0F2E48005D1209919B90999002900F014
:108A3000DD80002A00F34D81089A3B7007F10108A0
:108A40009742454600F05481214600230A224846B9
:108A500000F036FC5E45044631464FF000034FF00F
:108A60000A0248460BD000F02BFC5946064600236C
:108A70000A22484600F024FC47468346A6E700F059
:108A80001FFC474606468346A0E701464846059335
:108A900000F00CFC0122059BC0E74146204600F097
:108AA000E7FD0028BFF67DAD2146049C0023013C74
:108AB0000A224846049400F003FC099B0446002B5C
:108AC0007FF460AF0D9B002B40F3F681069370E5B9
:108AD000089C1FE5209B022B7FF767AD069B002BB0
:108AE00040F0798141460522484600F0E9FB014605
:108AF0008046204600F0BCFD002808947FF70EAFAA
:108B0000049A07993123013204920B704D1C09E736
:108B1000049A01320492079A3123137088E50123E5
:108B20000993CDE5DDF8149091E4BAF1000F7FF4DC
:108B300004ADCBF31303002B40F03F812BF0004733
:108B40003F0D3F0537B1059B01330593029B013370
:108B5000029301270B9B0120002B3FF4F8ACEDE4BE
:108B60004046FCF70BFC32463B46FCF76DFC00220E
:108B7000BF4BFCF7B7FA0446A1F1507530463946B1
:108B80000022BC4BFCF7ACFA22462B4606460F46A9
:108B9000FCF7EAFE8046002840F00581224605F1F8
:108BA000004330463946FCF7C1FE08B14646B5E6FB
:108BB000DDE90EABFFF789BB0798FFF7AEBA0A9B5A
:108BC0000B9A0A97FB1A1A440B92002761E4DDE91D
:108BD0000EAB4FF00208BBE51C460021C9F844105B
:108BE0008AE5012421940D940694F6E7002AD046E4
:108BF000CDF814B09A4611DD21460122484600F016
:108C0000DFFC4146044600F033FD002840F3498173
:108C1000BAF1390F00F0068105F1310AB34687F841
:108C200000A07D1C059E089402E504D11AF0010FF6
:108C300001D0EDE4154615F8013C302B05F1FF326B
:108C4000F8D0F5E4049B5C42002C00F0BF808A4B16
:108C500004F00F0203EBC203D3E90023DDE90E01A8
:108C6000FCF7F2FB241106460F4600F02A81834DE3
:108C70004FF00208E20709D530463946D5E900230E
:108C8000FCF7E2FB08F1010806460F46641005F107
:108C90000805EFD176E5079930220A70049A15F895
:108CA000014C01320492FFF7D0BB7168484600F0D6
:108CB000D7FA33699A1C0546920006F10C010C3074
:108CC000FAF790FD29460122484600F079FC05900C
:108CD00070E6392BCDF814B0D04600F0A38003F134
:108CE000010AB34687F800A07D1C059E08949FE406
:108CF0005A46D046B3469A4616467DE45E4908F188
:108D0000FF3A01EBCA0122462B46D1E90001FCF7EC
:108D10009BFBCDE912013946304600F05FFE044668
:108D2000FCF72CFB02460B4630463946FCF7D8F9D7
:108D3000079A3034B8F1010F06460F46147002F15D
:108D400001051ED0079B03EB080BA84600224C4BE5
:108D500030463946FCF778FB0F46064600F03EFEEB
:108D60000446FCF70BFB303402460B4630463946CE
:108D7000FCF7B6F908F8014BC34506460F46E5D1A6
:108D8000554400223F4BDDE91201FCF7ABF93246B6
:108D90003B46FCF7CBFD00284CD0119B049315F803
:108DA000014CFFF746BB4FF000084646A8E6059B7E
:108DB000069A9D1A0023FFF772BB0027CAE6149B90
:108DC0000A9F059DC3F13603FFF769BBDDE90E6716
:108DD0004FF00208D6E40894A0E5069B002B3FF470
:108DE000BFAE0D9B002B7FF7E3AE0022244B304635
:108DF0003946FCF729FB06460F4608F10100FCF74F
:108E0000BDFA32463B46FCF71FFB0022184BFCF72D
:108E100069F9049ADDF83480013A0446A1F15075ED
:108E20001192D0E43922B3460894059E3A707D1C15
:108E3000FFF7F0BBDDE9122300201249FCF750F9DF
:108E400032463B46FCF790FD08B9B1E6154615F8E9
:108E5000013C302B05F1FF32F8D030E5119B049333
:108E6000FFF7E7BABAF1000F7FF47AAD61E600BF11
:108E700000001C4000001440A0A4000078A50000E1
:108E8000000024400000E03F392BCDF814B0D0465C
:108E9000DDF808B09A46C5D0BBF1000F3FF7BCAE75
:108EA000BCE67FF4BBAE1AF0010F3FF4B7AEAFE6FD
:108EB0004FF00008464631E5209B022B21DC0D9B3C
:108EC00004E64FF002085DE4209B022B19DC0D9BA9
:108ED00063E50024C9F844402146484600F0C0F943
:108EE0004FF0FF3306930D93012307902194C9F8A7
:108EF00040000993FFF7E9B93FF43DABC0F13C00F6
:108F000022E50D9B0693E9E50125FFF7A8B900BF0F
:108F100038B5074D074C2C1BA41005D0013C55F863
:108F2000043D9847002CF9D1BDE8384001F048BB1A
:108F30000000000000000000F8B5234F0C46064674
:108F4000FDF72CF9BB685D6825F00305291B01F6C8
:108F5000EF7121F47F6121F00F01A1F58054B4F588
:108F6000805F07DB00213046FDF70CFBBB682B441C
:108F7000984204D03046FDF713F90020F8BD614255
:108F80003046FDF7FFFA01300DD0104BBA68196872
:108F90002D1B45F001053046091B55601960FDF792
:108FA000FFF80120F8BD00213046FDF7EBFABA6862
:108FB000831A0F2BDEDD064C0449246843F00103BD
:108FC000001B53600860D5E7D0A0FF1F00030020FE
:108FD000DCA4FF1F002945D02DE9F0410D46804655
:108FE000FDF7DCF855F8047C6A4927F00103A5F188
:108FF0000804E2188E685068B24220F0030062D084
:10900000FE0750600BD455F8087CE41B01F1080EF4
:10901000A56875453B446FD0E768EF60BD601518E3
:109020006D68ED0742D543F001026260E350B3F58D
:10903000007F18D2DB085A1C4D6851F83270A760C7
:1090400001209B1000FA03F301EBC2001D43083816
:10905000E0604D6041F83240FC604046BDE8F041C0
:10906000FDF79EB870475A0A042A53D89A0902F1AC
:1090700039077F0002F1380501EB870051F82720FE
:109080004449083890424DD0516821F003018B4289
:1090900002D292689042F7D1D068E060A26084600A
:1090A000D4604046BDE8F041FDF77AB895683A4F84
:1090B000BD4203443FD0D068E86043F001028560C0
:1090C0006260E350B3E7FF07034407D455F8082C68
:1090D000A41A1344A068E268C26090602F4A126824
:1090E00043F00100934260608C60B6D32C4B404645
:1090F0001968FFF721FFB0E711184968C90744D480
:109100009168D268CA60034443F0010091606060D6
:10911000E350A2E7142A17D802F15C077F0002F19E
:109120005B05A9E7AA104B68012505FA02F2134373
:109130004B600246B1E743F001024C610C61E5600F
:10914000A5606260E35088E7542A06D81A0B02F142
:109150006F077F0002F16E058EE7B2F5AA7F06D891
:10916000DA0B02F178077F0002F1770584E740F21D
:109170005450824206D89A0C02F17D077F0002F11A
:109180007C0579E7FE277E2576E743F001026260E1
:10919000E35062E7D0A0FF1FD8A0FF1FD8A4FF1F95
:1091A000FC020020044A054B1268506B002808BFDF
:1091B0001846F030704700BF609FFF1F649FFF1F7D
:1091C00001F0FF01102A2BDB10F0070F08D010F878
:1091D000013B013A8B422DD010F0070F42B3F6D17C
:1091E000F0B441EA012141EA014122F007047FF095
:1091F00000070023F0E80256083C85EA010586EAEC
:10920000010685FA47F5A3FA87F586FA47F6A5FA27
:1092100087F68EB9EED1F0BC01F0FF0102F0070233
:1092200032B110F8013B013A83EA010313B1F8D1DE
:109230000020704701387047002D06BF35460338BF
:10924000073815F0010F07D1013015F4807F02BFF8
:10925000013015F4C03F0130F0BC0138704700BF49
:10926000C36C70B505460C464BB153F8240080B171
:10927000026843F8242000230361C36070BD2122EB
:109280000421FCF797FBE86403460028EDD1002099
:1092900070BD012101FA04F6721D28469200FCF708
:1092A00089FB0028F3D044608660E4E731B1C36CE9
:1092B0004A6853F82200086043F82210704700BF44
:1092C000F0B50C6983B00D46064601F1140E002777
:1092D000DEF8000081B202FB01310B0C000C02FB36
:1092E000003389B2013701EB0341BC424EF8041B45
:1092F0004FEA1343ECDC3BB1AA68944207DA05EB72
:109300008402013453612C61284603B0F0BD6968C2
:10931000019301313046FFF7A3FF2A69023205F1BC
:109320000C01074692000C30FAF75CFAF26C69689F
:10933000019B52F82100286042F821503D46DEE7AB
:10934000030C1B04B3B90004102310F07F4F04BFBB
:109350000002083310F0704F04BF0001043310F016
:10936000404F04BF80000233002807DB420003D4D3
:10937000202070470023E8E7581C704718467047C4
:10938000036813F0070207D0D90720D49A0720D426
:109390009B0803600220704799B209B91B0C102288
:1093A00013F0FF0F04BF1B0A0832190704BF1B0983
:1093B0000432990704BF9B080232D90704D45B0822
:1093C00001D1202070470132036010467047002011
:1093D00070475B0803600120704700BF10B50C4662
:1093E0000121FFF73DFF01224461026110BD00BF72
:1093F0002DE9F04F0D691769BD4283B00C46164642
:1094000004DA2A4634463D460E461746A36861688C
:1094100005EB07089845C8BF0131FFF721FF00F1B0
:10942000140C0CEB8809CC45009005D26346002152
:1094300043F8041B9945FBD806F1140202EB870A96
:1094400004F11403524503EB850E54D2CDF8049079
:10945000994652F8043B1FFA83FBBBF1000F20D062
:1094600000204F466646054600E01E4657F8044B6E
:109470003068A1B283B20BFB0131240C000C4B19F4
:109480000BFB040000EB134099B2334641EA004164
:10949000BE454FEA104543F8041BE6D8756052F804
:1094A000043C5FEA134B20D0DCF8003067461846D6
:1094B0004D46002100E037462C88000C0BFB0400D1
:1094C00001449CB23E4644EA014346F8043B7868B6
:1094D00055F8044B83B2240C0BFB043404EB11430A
:1094E000AE454FEA1341E6D87B6092450CF1040C7F
:1094F000AFD8DDF80490B8F1000F0BDD59F8043C4B
:10950000A9F104091BB105E059F8043D13B9B8F1FC
:109510000108F9D10098C0F8108003B0BDE8F08FC1
:1095200012F003032DE9F041144607462ED10E46F2
:10953000A4101CD0BD6C95B3E3074FF0000806D40F
:10954000641014D02868A8B10546E307F8D52A4668
:1095500031463846FFF74CFFB6B17268FB6C6410B9
:1095600053F82210316043F822600646EAD13046B3
:10957000BDE8F0812A4629463846FFF739FF2860C2
:10958000C0F800800546E0E70646D9E75A1E0B4DB5
:10959000002355F82220FFF793FE0646C8E7012175
:1095A0003846FFF75DFE40F2712101220023416140
:1095B00002610546B8640360BEE700BF68A500000D
:1095C0002DE9F04791460A698B684FEA691404EB6C
:1095D000020808F101059D420E468246496804DDF5
:1095E0005B009D4201F10101FADC5046FFF738FEB5
:1095F000002C00F1140238DD02EB8403002142F854
:10960000041B9342FBD1346906F1140119F01F09C0
:1096100001EB840E21D0C9F1200200240F6807FA63
:1096200009FC4CEA04049C4643F8044B51F8044BF3
:109630008E4524FA02F4F1D8CCF804400CB108F1BC
:109640000205DAF84C307268013D53F822100561CA
:10965000316043F82260BDE8F087043B51F8042BE9
:1096600043F8042F8E45F9D8EBE71346CBE700BF4C
:1096700002690B69D21A12D19B00143014311944BB
:1096800010B4034401E098420BD253F8044D51F852
:10969000042D9442F7D007D3012010BC7047104628
:1096A0007047002010BC70474FF0FF30F5E700BF57
:1096B0002DE9F8430B690F4611695B1A002B9046A0
:1096C00017D1890007F1140208F114055318294431
:1096D00001E09A425ED253F8046D51F8044DA6425F
:1096E000F7D060D23B46144647464FF001099846F2
:1096F00006E05DDB07F1140502F114044FF00009E8
:109700007968FFF7ADFDD8F810303E69C0F80C90CD
:1097100004EB830CA64605EB860700F11404002336
:109720005EF8041B55F8048B8AB213FA88F3090C0F
:109730009A1AC1EB184303EB224392B242EA034266
:10974000F44544F8042B4FEA2343E9D8AF4217D934
:10975000A446294651F804EB13FA8EF2131403EBD6
:109760001E4392B242EA03428F424CF8042B4FEA66
:109770002343EFD8ED433D4425F0030504352C4445
:10978000043C22B954F8043D013E002BFAD0066196
:10979000BDE8F8830021FFF763FD01220023026189
:1097A0004361BDE8F8832C464FF000091546A7E752
:1097B0003B4607F1140408F1140547464FF0010930
:1097C00098469DE72DE9F04182B001211C46C3F384
:1097D0000A571546089EFFF743FDC4F3130480465D
:1097E0000FB144F4801401941DB302A840F8085D41
:1097F000FFF7C6FD002834D19DE80C00C8F81420FE
:10980000002B0CBF01210221C8F81830C8F8101035
:10981000DFB908EB8103A0F2324030601869FFF72E
:109820008FFD099BC0EB41101860404602B0BDE8B7
:10983000F08101A8FFF7A4FD019BC8F814300121B5
:109840002030C8F81010002FE3D0099BA7F233474F
:109850000744C0F1350037601860404602B0BDE8EB
:10986000F0819DE80C00C0F1200103FA01F10A43E8
:10987000C3400193C8F81420C2E700BF2DE9F04FA0
:10988000936883B09046002B72D083464FF0000956
:10989000166808688B680D464C46002C45D09C42E3
:1098A0001F469A4646D3AB8913F4906F2DD06F694B
:1098B000296907EB4707C1EB000A07EBD777601C64
:1098C0007F105044B8423A4684BF07463A465B058B
:1098D00033D511465846FCF7E1F8002837D05246F8
:1098E00029690190F9F77EFFAA89019B22F4906211
:1098F00042F08002AA81CAEB070203EB0A006F6103
:109900002B612860AA602746A24652464946FCF7CA
:1099100093FBD8F80820AB682868DB1B5044141B65
:10992000AB602860C8F8084014B3D6F8009074689B
:109930000836B2E72746A246E7E75846FCF732FC6E
:1099400003460028D7D129695846FFF743FB0C236B
:10995000CBF80030AB89002243F040034FF0FF30DA
:10996000AB81C8F80820C8F8042003B0BDE8F08F28
:109970000020C8F8040003B0BDE8F08F70B51546AC
:109980009AB0146809B1002C1AD100244FF4227245
:10999000ADF80C20009404941A464FF6FF761E9BF7
:1099A000029469460594ADF80E60FCF797FE002816
:1099B00011DB009B286000221A7004981AB070BD59
:1099C0004FF4C16200910491ADF80C20E4DA8B23CE
:1099D00003600020F2E70020F0E700BF4FEA4102F9
:1099E00012F5001215D211D56FF47873B3EB6252F1
:1099F00012D94FEAC12343F0004343EA505311F018
:109A0000004F23FA02F018BF404270474FF00000A9
:109A1000704750EA013005D111F0004008BF6FF0E7
:109A2000004070474FF00000704700BF53B94AB97B
:109A3000002908BF00281CBF4FF0FF314FF0FF3056
:109A400000F07EB9ADF1080C6DE904CE00F006F827
:109A5000DDF804E0DDE9022304B070472DE9F047AA
:109A60008C460E460446089D002B50D18A4217466C
:109A70006CD9B2FA82FEBEF1000F0BD0CEF12004F9
:109A800020FA04F401FA0EF644EA060C02FA0EF784
:109A900000FA0EF44FEA1749220CBCFBF9F01FFA4A
:109AA00087F809FB10C642EA064600FB08F3B342FA
:109AB00009D9F61900F1FF3280F02281B34240F259
:109AC0001F8102383E44F61AA2B2B6FBF9F309FB35
:109AD000136642EA064403FB08F8A04509D9E419D5
:109AE00003F1FF3280F00A81A04540F20781023B7A
:109AF0003C44C8EB040443EA00400021002D62D03E
:109B000024FA0EF400232C606B60BDE8F0878B42D2
:109B100007D9002D55D0002185E841000846BDE851
:109B2000F087B3FA83F1002940F09080B34202D36A
:109B3000824200F2F880841A66EB03060120B446E4
:109B4000002D40D085E81010BDE8F08712B901273C
:109B5000B7FBF2F7B7FA87FEBEF1000F35D1F31B62
:109B60004FEA17481FFA87FC0121B3FBF8F0220CDB
:109B700008FB103642EA06460CFB00F3B34207D955
:109B8000F61900F1FF3202D2B34200F2CE80104645
:109B9000F61AA2B2B6FBF8F308FB136642EA0644D3
:109BA0000CFB03FCA44507D9E41903F1FF3202D2F0
:109BB000A44500F2B5801346CCEB040443EA004010
:109BC0009CE729462846BDE8F087CEF1200106FA39
:109BD0000EF307FA0EF720FA01F94FEA1748CE40C4
:109BE00049EA0309B6FBF8FA4FEA194408FB1A667A
:109BF0001FFA87FC44EA06430AFB0CF29A4200FA79
:109C00000EF40AD9DB190AF1FF3180F087809A42FD
:109C100040F28480AAF1020A3B449B1A1FFA89F998
:109C2000B3FBF8F108FB113349EA034301FB0CF6DF
:109C30009E4207D9DB1901F1FF326BD29E4269D9EE
:109C400002393B449B1B41EA0A418EE7C1F1200ED9
:109C500022FA0EF48B40234320FA0EF706FA01F4A1
:109C60004FEA134C26FA0EF63C43B6FBFCF9270CE0
:109C70000CFB19661FFA83F847EA064609FB08F74A
:109C8000B74202FA01F200FA01FA08D9F61809F10E
:109C9000FF3041D2B7423FD9A9F102091E44F61B59
:109CA000A0B2B6FBFCF40CFB146640EA064704FBCA
:109CB00008F8B84507D9FF1804F1FF3028D2B84595
:109CC00026D9023C1F4444EA0940C8EB0707A0FB21
:109CD00002894F4544464E4614D329D065B3BAEBAA
:109CE000040367EB060707FA0EFECB40CF404EEAAF
:109CF000030385E888000021BDE8F0871346F8E6F5
:109D00001046E0E6B8EB020469EB03060138E5E72C
:109D10000446D8E7114695E78146C0E78A467CE7C6
:109D2000023B3C4448E708460AE702383E442FE736
:109D3000C245E7D33E46D1E72946BDE8F08700BFDC
:109D4000704700BF7573625F7365747570205479D6
:109D500070652025780D0A004441432042617365F7
:109D60006C696E652025640D0A00000054584C652E
:109D700076656C202564203D202564206D5600000A
:109D800052584C6576656C202564203D2025642062
:109D90006D560000727473203D2025640A00000097
:109DA000647472203D2025640A0000000D0A000042
:109DB00075706461746520636F756E74202564200E
:109DC000666C616720256400000000000000000050
:109DD00075080000990800002D09000029090000FD
:109DE00025090000210900001D090000E908000004
:109DF000FD080000E5080000DD080000D5080000AF
:109E0000CD080000BD080000AD080000A908000052
:109E1000ED070000F5070000FD0700000508000041
:109E2000810800006908000025732025690D0A00DB
:109E300041646A757374696E67205258204C657668
:109E4000656C202564206D5620506F7420256400B9
:109E500041646A757374696E67205458204C657646
:109E6000656C202564206D5620506F742025640099
:109E70004D6F6E69746F722042756666657220530D
:109E8000706163652025640D0A000000486F7374DB
:109E90002042756666657220537061636520256493
:109EA000000000000A2A2A2A2A20526573657420BD
:109EB0006279205761746368646F67202B2B2B2BAA
:109EC0000000000053616D706C6520526174652064
:109ED00025642050444220446976696465722025D7
:109EE000640000005258204C6576656C20666978E5
:109EF0006564206174202564200000004C6576654F
:109F00006C2062656C6F77207468726573686F6C23
:109F100064202D20617373756D65206E6F20696EEE
:109F200070757420256420256420256420706B00E2
:109F30007065616B20746F207065616B20696E7055
:109F40007574202564206D5600FFFFFF496E707503
:109F500074207065616B7320256420256420617610
:109F6000657261676520256400000000494E505508
:109F7000545045414B5320256420256400000000C7
:109F8000746F7453616D706C657320256400FFFFFE
:109F90000000000000000000A9120000D51200001F
:109FA000E9070000A51200004D1200005D1200003C
:109FB00085120000696E20496E7473202564204F5D
:109FC000757420696E7473202564205120256420E7
:109FD000746F7420727820256420746F74207478F4
:109FE0002025642071756575656420256400000076
:109FF0007365742066656174757265202578202507
:10A000007820257820257820257820257820257827
:10A01000202578202578202578202578202578206F
:10A0200025782025780000006765742066656174D6
:10A0300075726520257820257820257820257820C0
:10A04000257820257800FFFF151915151914181407
:10A05000000100001C98FF1F120000000002000019
:10A060004898FF1F35010000002202008099FF1F61
:10A070001C000000002102009C98FF1F0900000046
:10A0800000030000D499FF1F000000000103090431
:10A090003098FF1F00000000020309049C99FF1F75
:10A0A0000000000003030904D899FF1F000000000E
:10A0B0000000000000000000000000004745545F61
:10A0C000435552003C80044000100000041A000078
:10A0D000FF7F000011100000AD2C00000C080000F4
:10A0E00000020000000200000B0700004002000018
:10A0F000000200000D0E00004002000000020000FF
:10A100000A020906141715160F00000000020000CD
:10A110000002000000020000000200000002000037
:10A120000002000000020000000200000002000027
:10A1300001010202040408081000000000000000F1
:10A14000000000003D31000061310000F5310000E9
:10A15000F1310000ED310000E9310000E53100008F
:10A16000B1310000C5310000AD310000A531000063
:10A170009D310000953100008531000075310000EF
:10A1800071310000193200003932000059320000EC
:10A19000F931000049310000313100000D0AFFFFA4
:10A1A000050E08090D0C06070F0400130393050E96
:10A1B00008090D0C06070F04FFFFC585848687C4B8
:10A1C000FFFF001303931A9217FFFFFF6FF07F0347
:10A1D0000370037813F0800FFBD070474008FE43F4
:10A1E00040A004404408FE4344A004400018FE433D
:10A1F00000C004403000FE43309004403400FE4371
:10A20000349004401C18FE431CC004401018FE4348
:10A2100010C004400818FE4308C004400C18FE4358
:10A220000CC004400C10FE430CB004401010FE4360
:10A2300010B004401810FE4318B004401C10FE4338
:10A240001CB004401410FE4314B004400418FE4334
:10A2500004C004400010FE4300B004400008FE4368
:10A2600000A004400408FE4304A004400C08FE4380
:10A270000CA004400808FE4308A004401418FE4344
:10A2800014C004401818FE4318C004400410FE43D4
:10A2900004B004400810FE4308B004401400FE431C
:10A2A000149004404C08FE434CA004400420FE439C
:10A2B00004D004402410FE4324B004402010FE4388
:10A2C00020B004402810FE4328B004402C10FE4368
:10A2D0002CB004400020FE4300D004404808FE4358
:10A2E00048A004401000FE4310900440000000000D
:10A2F00000000000014B0000F94A0000F54A000090
:10A30000F14A0000ED4A0000E94A0000E54A000079
:10A31000E14A0000389BFF1F43000000504F5349A3
:10A32000580000002E00FFFF303030303030303029
:10A330003030303030303030494E4600696E660083
:10A340004E414E006E616E00303132333435363757
:10A350003839414243444546000000003031323331
:10A360003435363738396162636465660000000051
:10A37000286E756C6C2900003000FFFF2020202023
:10A3800020202020202020202020202000202020ED
:10A390002020202020202828282828202020202095
:10A3A0002020202020202020202020202088101065
:10A3B00010101010101010101010101010040404C1
:10A3C000040404040404041010101010101041417F
:10A3D000414141410101010101010101010101016D
:10A3E0000101010101010101101010101010424281
:10A3F000424242420202020202020202020202023D
:10A4000002020202020202021010101020000000DC
:10A41000000000000000000000000000000000003C
:10A42000000000000000000000000000000000002C
:10A43000000000000000000000000000000000001C
:10A44000000000000000000000000000000000000C
:10A4500000000000000000000000000000000000FC
:10A4600000000000000000000000000000000000EC
:10A4700000000000000000000000000000000000DC
:10A4800000000000000000000000000000FFFFFFCF
:10A49000496E66696E697479000000004E614E0075
:10A4A000000000000000F03F000000000000244019
:10A4B00000000000000059400000000000408F40F4
:10A4C000000000000088C34000000000006AF8405F
:10A4D0000000000080842E4100000000D012634183
:10A4E0000000000084D797410000000065CDCD41F9
:10A4F000000000205FA00242000000E876483742DA
:10A50000000000A2941A6D42000040E59C30A24277
:10A510000000901EC4BCD64200003426F56B0C43EC
:10A520000080E03779C3414300A0D8855734764393
:10A5300000C84E676DC1AB43003D9160E458E143F4
:10A54000408CB5781DAF154450EFE2D6E41A4B4469
:10A5500092D54D06CFF08044F64AE1C7022DB544AE
:10A56000B49DD9794378EA44050000001900000041
:10A570007D000000FFFFFFFF0080E03779C341430B
:10A58000176E05B5B5B89346F5F93FE9034F384D59
:10A59000321D30F94877825A3CBF737FDD4F157505
:10A5A000F8B500BFF8BC08BC9E467047717F00003C
:10A5B00035040000C507000081100000DD1900000F
:04A5C000F8B500BF2B
:08A5C40098F4FF7F0100000084
:10A5CC0038B5084B1C681C6054B1074D94FAA4F3C1
:10A5DC00B3FA83F355F823309847631E1C40F5D12A
:10A5EC0038BD00BFA0D00440189BFF1F38B5084BE6
:10A5FC001C681C6054B1074D94FAA4F3B3FA83F3AE
:10A60C0055F823309847631E1C40F5D138BD00BF68
:10A61C00A0C00440F89AFF1F38B5084B1C681C609A
:10A62C0054B1074D94FAA4F3B3FA83F355F82330DD
:10A63C009847631E1C40F5D138BD00BFA0B0044044
:10A64C00C89AFF1F38B5084B1C681C6054B1074DE5
:10A65C0094FAA4F3B3FA83F355F823309847631EA6
:10A66C001C40F5D138BD00BFA0A00440789AFF1F54
:10A67C0038B5084B1C681C6054B1074D94FAA4F310
:10A68C00B3FA83F355F823309847631E1C40F5D179
:10A69C0038BD00BFA0900440409AFF1F000000008E
:10A6AC0000000C0080000000FF0000000080000093
:10A6BC00D09D000000000000E80300000000000036
:10A6CC000100000028DAFF1F006006400160064010
:10A6DC0002600640036006400460064005600640C8
:10A6EC0006600640076006400860064009600640A8
:10A6FC000A6006400B6006400000000000000000ED
:10A70C00000000000000000000000000000000003D
:10A71C00000000000000000000000000000000002D
:10A72C00000000000000000000000000000000001D
:10A73C00000000000000000000000000000000000D
:10AB0C00000000000000000001000100A086010010
:10AB1C000100000000000000000000000000000028
:10AB2C000000000000000000000000000070064063
:10AB3C000170064002700640037006400470064027
:10AB4C000570064006700640077006400870064007
:10AB5C00097006400A7006400B70064000000000A9
:10AB6C0000000000000000000000000000000000D9
:10AB7C0000000000000000000000000000000000C9
:10AB8C0000000000000000000000000000000000B9
:10AB9C0000000000000000000000000000000000A9
:10AF6C0000000000000000000000000001000200D2
:10AF7C00A08601000100000000000000000000009D
:10AF8C0000000000000000000000000000000000B5
:10AF9C00000000000000000019000000000000008C
:10AFAC00000000000000000080BB00001201100136
:10AFBC0000000040C0168A04750201020301000063
:10AFCC0018035400650065006E007300790064007E
:10AFDC00750069006E006F0009023501060100C0A2
:10AFEC0032080B00020202010409040000010202F3
:10AFFC0001000524001001052401010104240206AE
:10B00C000524060001070581031000400904010016
:10B01C00020A000000070502024000000705830237
:10B02C004000000904020002030000000921110184
:10B03C000001221C000705840340000107050503DD
:10B04C00400001080B030301010000090403000088
:10B05C00010100000A2401000148000204050C242F
:10B06C00020103060002030000000A24063101015C
:10B07C00030000000924030201010031000C24022A
:10B08C000301010002030000000A2406320301033D
:10B09C000000000924030403060032000904040024
:10B0AC000001020000090404010101020000072450
:10B0BC0001020301000B2402010202100180BB00FB
:10B0CC0009058605C00001000007250100000000ED
:10B0DC000904050000010200000904050102010237
:10B0EC000000072401030301000B240201020210DB
:10B0FC000180BB0009050705C00001008807250178
:10B10C000000000009058811030001050000000083
:10B11C0006ABFF0A0002A1017508150026FF009579
:10B12C004009018102954009029102C03603540086
:10B13C00650065006E007300790020004100750009
:10B14C00640069006F002F005300650072006900F5
:10B15C0061006C002F00520061007700480049002C
:10B16C0044000000040309040C030000000000006C
:10B17C0000000000000000000000000000000000C3
:10B18C0000C00240C4A0000000000000000000004D
:10B19C0000000000000000000000000000000000A3
:10B1AC000000000000000000000000000000000093
:10B1BC00000000000000000044A10000000000009E
:10B1CC00E8030000000000000A0400005C030020FB
:10B1DC00313A0000313A0000313A0000313A0000B7
:10B1EC00313A0000313A0000313A0000313A0000A7
:10B1FC00313A0000313A0000313A0000313A000097
:10B20C00313A0000313A0000313A0000313A000086
:10B21C00313A0000313A0000313A0000313A000076
:10B22C00313A0000313A0000313A0000313A000066
:10B23C00313A0000313A0000313A0000313A000056
:10B24C00313A0000313A0000313A0000313A000046
:10B25C00313A0000313A0000313A0000313A000036
:10B26C00313A0000313A0000313A0000313A000026
:10B27C00313A0000313A0000313A0000313A000016
:10B28C00313A0000313A0000313A0000313A000006
:10B29C00313A0000313A0000313A0000313A0000F6
:10B2AC00313A0000313A0000313A0000313A0000E6
:10B2BC0001080000F4A2000000000000E8030000F8
:10B2CC0000000000FFFFFFFF00000000249EFF1F96
:10B2DC008C9EFF1FF49EFF1F00000000000000006A
:10B2EC000000000000000000000000000000000052
:10B2FC000000000000000000000000000000000042
:10B30C000000000000000000000000000000000031
:10B31C000000000000000000000000000000000021
:10B32C000000000000000000000000000000000011
:10B33C000000000000000000000000000000000001
:10B34C0000000000000000000000000000000000F1
:10B35C0000000000000000000000000000000000E1
:10B36C0000000000000000000000000000000000D1
:10B37C0001000000000000000E33CDAB34126DE66E
:10B38C00ECDE05000B0000000000000000000000D7
:10B39C0000000000000000000000000000000000A1
:10B3AC000000000000000000000000000000000091
:10B3BC000000000000000000000000000000000081
:10B3CC000000000000000000000000000000000071
:10B6FC00389BFF1F4300000000000000000000000A
:10B70C00000000000000000000000000000000002D
:10B71C0000000000430000000000000000000000DA
:10B72C00000000000000000000000000000000000D
:10B73C0000000000430000000000000000000000BA
:10B74C0000000000000000000000000000000000ED
:10B75C00000000004300000000000000000000009A
:10B76C0000000000000000000000000000000000CD
:10B77C00000000004300000000000000000000007A
:10B78C0000000000000000000000000000000000AD
:10B79C00000000004300000000000000000000005A
:10B7AC00000000000000000000000000000000008D
:10B7BC00000000004300000000000000000000003A
:10B7CC00000000000000000000000000000000006D
:10B7DC0000000000857E00000D60000000000000ED
:10B7EC008CA3000024A30000C09E0000C09E00009B
:10B7FC00C09E0000C09E0000C09E0000C09E0000C5
:10B80C00C09E0000C09E0000C09E0000FFFFFFFF16
:10B81C00FFFFFFFFFFFFFFFFFFFF00000100415391
:10B82C004349490000000000000000000000000037
:10B83C000000000000000000000000000000415368
:10B84C004349490000000000000000000000000017
:10B85C0000000000000000000000000000000000DC
:10B86C000000000000000000D0A0FF1FD0A0FF1FB0
:10B87C00D8A0FF1FD8A0FF1FE0A0FF1FE0A0FF1F54
:10B88C00E8A0FF1FE8A0FF1FF0A0FF1FF0A0FF1F04
:10B89C00F8A0FF1FF8A0FF1F00A1FF1F00A1FF1FB2
:10B8AC0008A1FF1F08A1FF1F10A1FF1F10A1FF1F60
:10B8BC0018A1FF1F18A1FF1F20A1FF1F20A1FF1F10
:10B8CC0028A1FF1F28A1FF1F30A1FF1F30A1FF1FC0
:10B8DC0038A1FF1F38A1FF1F40A1FF1F40A1FF1F70
:10B8EC0048A1FF1F48A1FF1F50A1FF1F50A1FF1F20
:10B8FC0058A1FF1F58A1FF1F60A1FF1F60A1FF1FD0
:10B90C0068A1FF1F68A1FF1F70A1FF1F70A1FF1F7F
:10B91C0078A1FF1F78A1FF1F80A1FF1F80A1FF1F2F
:10B92C0088A1FF1F88A1FF1F90A1FF1F90A1FF1FDF
:10B93C0098A1FF1F98A1FF1FA0A1FF1FA0A1FF1F8F
:10B94C00A8A1FF1FA8A1FF1FB0A1FF1FB0A1FF1F3F
:10B95C00B8A1FF1FB8A1FF1FC0A1FF1FC0A1FF1FEF
:10B96C00C8A1FF1FC8A1FF1FD0A1FF1FD0A1FF1F9F
:10B97C00D8A1FF1FD8A1FF1FE0A1FF1FE0A1FF1F4F
:10B98C00E8A1FF1FE8A1FF1FF0A1FF1FF0A1FF1FFF
:10B99C00F8A1FF1FF8A1FF1F00A2FF1F00A2FF1FAD
:10B9AC0008A2FF1F08A2FF1F10A2FF1F10A2FF1F5B
:10B9BC0018A2FF1F18A2FF1F20A2FF1F20A2FF1F0B
:10B9CC0028A2FF1F28A2FF1F30A2FF1F30A2FF1FBB
:10B9DC0038A2FF1F38A2FF1F40A2FF1F40A2FF1F6B
:10B9EC0048A2FF1F48A2FF1F50A2FF1F50A2FF1F1B
:10B9FC0058A2FF1F58A2FF1F60A2FF1F60A2FF1FCB
:10BA0C0068A2FF1F68A2FF1F70A2FF1F70A2FF1F7A
:10BA1C0078A2FF1F78A2FF1F80A2FF1F80A2FF1F2A
:10BA2C0088A2FF1F88A2FF1F90A2FF1F90A2FF1FDA
:10BA3C0098A2FF1F98A2FF1FA0A2FF1FA0A2FF1F8A
:10BA4C00A8A2FF1FA8A2FF1FB0A2FF1FB0A2FF1F3A
:10BA5C00B8A2FF1FB8A2FF1FC0A2FF1FC0A2FF1FEA
:10BA6C00C8A2FF1FC8A2FF1FD0A2FF1FD0A2FF1F9A
:10BA7C00D8A2FF1FD8A2FF1FE0A2FF1FE0A2FF1F4A
:10BA8C00E8A2FF1FE8A2FF1FF0A2FF1FF0A2FF1FFA
:10BA9C00F8A2FF1FF8A2FF1F00A3FF1F00A3FF1FA8
:10BAAC0008A3FF1F08A3FF1F10A3FF1F10A3FF1F56
:10BABC0018A3FF1F18A3FF1F20A3FF1F20A3FF1F06
:10BACC0028A3FF1F28A3FF1F30A3FF1F30A3FF1FB6
:10BADC0038A3FF1F38A3FF1F40A3FF1F40A3FF1F66
:10BAEC0048A3FF1F48A3FF1F50A3FF1F50A3FF1F16
:10BAFC0058A3FF1F58A3FF1F60A3FF1F60A3FF1FC6
:10BB0C0068A3FF1F68A3FF1F70A3FF1F70A3FF1F75
:10BB1C0078A3FF1F78A3FF1F80A3FF1F80A3FF1F25
:10BB2C0088A3FF1F88A3FF1F90A3FF1F90A3FF1FD5
:10BB3C0098A3FF1F98A3FF1FA0A3FF1FA0A3FF1F85
:10BB4C00A8A3FF1FA8A3FF1FB0A3FF1FB0A3FF1F35
:10BB5C00B8A3FF1FB8A3FF1FC0A3FF1FC0A3FF1FE5
:10BB6C00C8A3FF1FC8A3FF1FD0A3FF1FD0A3FF1F95
:10BB7C00D8A3FF1FD8A3FF1FE0A3FF1FE0A3FF1F45
:10BB8C00E8A3FF1FE8A3FF1FF0A3FF1FF0A3FF1FF5
:10BB9C00F8A3FF1FF8A3FF1F00A4FF1F00A4FF1FA3
:10BBAC0008A4FF1F08A4FF1F10A4FF1F10A4FF1F51
:10BBBC0018A4FF1F18A4FF1F20A4FF1F20A4FF1F01
:10BBCC0028A4FF1F28A4FF1F30A4FF1F30A4FF1FB1
:10BBDC0038A4FF1F38A4FF1F40A4FF1F40A4FF1F61
:10BBEC0048A4FF1F48A4FF1F50A4FF1F50A4FF1F11
:10BBFC0058A4FF1F58A4FF1F60A4FF1F60A4FF1FC1
:10BC0C0068A4FF1F68A4FF1F70A4FF1F70A4FF1F70
:10BC1C0078A4FF1F78A4FF1F80A4FF1F80A4FF1F20
:10BC2C0088A4FF1F88A4FF1F90A4FF1F90A4FF1FD0
:10BC3C0098A4FF1F98A4FF1FA0A4FF1FA0A4FF1F80
:10BC4C00A8A4FF1FA8A4FF1FB0A4FF1FB0A4FF1F30
:10BC5C00B8A4FF1FB8A4FF1FC0A4FF1FC0A4FF1FE0
:10BC6C00C8A4FF1FC8A4FF1F00000200FFFFFFFFB6
:00000001FF
